:106E86000000090200000301FA0400EF0500030AEE
:106E96000A5A0B001E0C00FA0D00030E00040F0127
:106EA60064100096120132130AFA14010217010A3D
:106EB6001801EF1905321A010A1B01EF1C05321FD2
:106EC600FFFF20FFFF23011E2400642A00FA2B0087
:106ED600FA2C50782D003D2E004630006432507852
:106EE6003300003432FA3501643601643701503814
:106EF6000A643A00033B00043C00643E003C3F0049
:106F06000140FFFF411450420A5A430AC844053261
:106F16004500B44600FA4900024B00014C00FA5005
:106F26000C0C510596520A32530B46540A965705D5
:106F360046590A465A32FA5B010A5C0A325E000A70
:106F46005F00646200FE64021067FFFF680101696A
:106F560001016A05966B00006C32966D00047300A1
:106F6600007400007801327901327E00647FFFFFF1
:106F760080FFFF8100008400648800028A00019D72
:106F86000A969E00019FFFFFA0FFFFA2000AA3FF33
:106F9600FFA4FFFFA5FFFFA6FFFFA7FFFFA8FFFFB8
:106FA600A9FFFF0101241500002F003C47012448DA
:106FB60002025602024EFFFF58000261FFFF660002
:106FC600018500AF8600018700FA89010499000057
:106FD600A100FAFAFAFA0065006F00790083008DC5
:106FE600009700A100AC00B600C000CA00D400DEC5
:106FF60000E800F200580060006800700078008029
:1070060000880090009800A000A800B000B800C159
:1070160000C800D000D800DF00E600EE00F6004110
:107026000047004D00530059005F0065006C007179
:107036000077007D00830089008F0095009B00A2E9
:1070460000A700AC00B200B900C000C500CA00D25B
:0A70560000D500DD00E100E700EFC7
:103CD80075A71085F97385FA747E017F00E5741263
:103CE8007172E5732FFF50010E8E598F5A90002480
:103CF800E0FCA3E0FDEF2DFDEE3CFC8C5B8D5C90C1
:103D08000044E0FAA3E0FBED2BFBEC3AFA8A5B8B6C
:103D18005C22E55CF5FBE55BF5FCD29322E55CF5FE
:103D2800E9E55BF5EAD29422E55CF5EBE55BF5ECB9
:103D3800D29122E55CF5EDE55BF5EED29222E55CE9
:103D4800F5FDE55BF5FED28722E55CF5CEE55BF592
:103D5800CFD29022E50C906A7BF82828738052A273
:103D680034B34008E5B54408F5B58006E5B554F721
:103D7800F5B5803DA234B34008E5B54440F5B580BB
:103D880006E5B554BFF5B58028A234B34008E5B5BB
:103D98004480F5B58006E5B5547FF5B58013A234A7
:103DA800B34008E5B54404F5B58006E5B554FBF520
:013DB800B555
:0F6A7B00023D65023D67023D7C023D91023DA652
:103DB90022743390017DF0743690017EF0742D9059
:103DC900017FF07432900180F07420900181F074C9
:103DD90031900182F07432900183F0744390018430
:103DE900F07479900185F0746C900186F0742090DC
:103DF9000187F07420900188F07420900189F07493
:103E09002090018AF0742090018BF0229008B4E090
:103E1900FEA3E0FF7423D39F74019E400C906E862D
:103E2900120048E493F59980129008B4E0FEA3E0EB
:103E3900FF906E86120048E493F5999008B41271C8
:103E4900809008B4E0FEA3E0FFEFB45607EEB4019A
:103E590003754D0022AE59AF5A740A8E048F05FFBF
:103E69001271628C5B8D5CAE59AF5A740A8E048FE5
:103E790005FF12718D8C598D5AE55A455960137495
:103E89000AC3955AFFE49559FE8E598F5A785B12E9
:103E990071C5E573A85BB80015D3955C4010E5734F
:103EA900C3955CFFE4955BFE8E5B8F5C8010E573C8
:103EB9002424C3955CFFE4955BFE8E5B8F5CAE5B4F
:103EC900AF5C74236F4E600674246F4E701AAE5B3C
:103ED900AF5C74236F4E70057573018003757302AF
:103EE900755C22755B008003757300229000BAE04F
:103EF900B40104C2068002D2069000BBE0B40104FA
:103F0900C2078002D2079000F8E075F0E1A4FFAE85
:103F1900F0740A8E048F05FF1271629008A8ECF004
:103F2900A3EDF09000F8E075F02BA4FFAEF090003F
:103F390020EEF0A3EFF07E017F009000B6E0127151
:103F4900729000F9E08E048F05FF127162740AFF06
:103F59001271628D60900102E075F0E1A4FFAEF08C
:103F6900740A8E048F05FF1271629008ACECF0A3FD
:103F7900EDF0900104E06013900104E0F5F074168F
:103F890084FF7E00EF90090AF08006746490090AA4
:103F9900F09000FAE0900098F0900148E0FE90005F
:103FA900F6E08E0088F0A4FFAEF0EF900913F090D0
:103FB9000121E075F013A4FDACF0900044ECF0A3EE
:103FC900EDF0A221B34016900192E0700C9001939C
:103FD900E07006900194E060028002C22190019293
:103FE900E0B4300F900193E0B44708900194E06485
:103FF9003B60028004D2228002C22274E3900097BF
:10400900F09000E3E0B40B0874E3900097F0805A55
:104019009000E3E0B419129000F9E0906FC7120024
:104029008CE493900097F080419000E3E0B41E1275
:104039009000F9E0906FE512008CE493900097F0FE
:1040490080289000E3E0B428129000F9E090700F06
:1040590012008CE493900097F0800F9000E3E0B495
:1040690046089000DAE0900097F09000B3E0FE90E7
:104079000914E06E601B7599E612019C74AB9000FF
:1040890071F012069A7464F5097508001205E48046
:10409900FE9000ABE0700674009000E0F090009C88
:1040A900E0FE9000E0E0B5063F90009EE0FE900043
:1040B900FEE0B5063390009DE0FE90010CE0B506E8
:1040C9002790009FE0FE9000B3E0B5061B9000A08A
:1040D900E0FE90012CE0B5060F9006EDE0FE9000A1
:1040E900A1E06E700302424C740790012FF090001A
:1040F900B3E0B4010674009000B3F09000B3E0B4EB
:10410900020674009000FEF09000B3E0B403067458
:104119000090010BF090010CE0B4012774009000AD
:10412900C8F0741C900132F074009006F4F0740029
:104139009006F5F09000E0E0B4020674019000E00A
:10414900F080339000E0E0B4021A741C9000C8F0CB
:104159007400900132F074009006F4F07400900637
:10416900F5F080127400900132F074009000C8F0EC
:10417900741C9006F4F09000FEE0D394014026747C
:10418900009000C7F0741B900131F074009006F0A4
:10419900F074009006F1F09000E0E0600674009081
:1041A90000E0F080329000E0E0601A741B9000C7D4
:1041B900F07400900131F074009006F0F0740090F2
:1041C90006F1F0801274009000C7F074009001317C
:1041D900F0741B9006F0F09006EDE0600874009012
:1041E90007A4F0800674299007A4F09000D3E0603A
:1041F900147409900136F074009006F8F074009078
:1042090006F9F0800C7400900136F074099006F8F4
:10421900F0D2209000E0E090009CF090010CE0903A
:10422900009DF09000FEE090009EF09000B3E090B9
:10423900009FF090012CE09000A0F09006EDE09036
:1042490000A1F09000A2E0FE9000D3E06E603E90E5
:1042590000D3E0600E7409900136F074009006F8FE
:10426900F0800C7400900136F074099006F8F09013
:1042790000A2E060069000D3E07002D2209000D343
:10428900E09000A2F09000D3E09008BEF0900116F3
:10429900E0B40117900030740FF0A374FFF09000A0
:1042A90032E4F0A3F07402900116F0900116E0B424
:1042B9000341900032E0FEA3E0FF900030E0FCA350
:1042C900E0FD1271BD74101271727408120039EF99
:1042D900900115F0EF700674FF900115F0740090CD
:1042E9000116F0900031E09000CCF0900030E090A1
:1042F90000CDF09000A7E09000A4F09000A6E09017
:1043090000A3F09000D5E0C3941E50569000D5E06C
:10431900F404241E9000A5F09000A5E075F00A842D
:10432900FF7E008F739000A5E075F00A84ADF07CE4
:10433900008D749000A3E0D39574400D9000A3E024
:10434900C395749000A3F0800F9000A3E0240AC3E2
:1043590095749000A3F005739000A4E02573900074
:10436900A4F09000A4E090005EF090005EE0D39489
:1043790024400B90005EE0C3942490005EF090000E
:104389005EE0240690005FF090005EE0240C90004F
:1043990060F090005EE02412900061F090005EE011
:1043A9002418900062F090005EE0241E900063F0F3
:1043B90090005FE0D39424400B90005FE0C3942405
:1043C90090005FF0900060E0D39424400B9000606F
:1043D900E0C39424900060F0900061E0D3942440FD
:1043E9000B900061E0C39424900061F0900062E0BA
:1043F900D39424400B900062E0C39424900062F0AF
:10440900900063E0D39424400B900063E0C39424AC
:10441900900063F090006AE4F090005EE06423602D
:104429000790005EE0B4242090005EE0B423067497
:104439000290006AF090005EE0B4240690006A746D
:1044490001F090005E7401F090006BE4F090005F61
:10445900E06423600790005FE0B4242090005FE0EF
:10446900B42306740290006BF090005FE0B4240658
:1044790090006B7401F090005F7401F090006CE49F
:10448900F0900060E064236007900060E0B42420AD
:10449900900060E0B42306740290006CF090006014
:1044A900E0B4240690006C7401F09000607401F08F
:1044B90090006DE4F0900061E06423600790006172
:1044C900E0B42420900061E0B42306740290006DEA
:1044D900F0900061E0B4240690006D7401F0900042
:1044E900617401F090006EE4F0900062E064236072
:1044F90007900062E0B42420900062E0B4230674BF
:104509000290006EF0900062E0B4240690006E7490
:1045190001F09000627401F090006FE4F090006384
:10452900E064236007900063E0B42420900063E016
:10453900B42306740290006FF0900063E0B424067F
:1045490090006F7401F09000637401F09000A7E08F
:10455900FE90010AE02E900072F0900072E0641261
:104569006007900072E0B42406900072E004F090B5
:104579000072E064116007900072E0B423069000B5
:1045890072E014F0900072E0D39424400B90007212
:10459900E0C39424900072F0900072E0D39412402A
:1045A9000D900072E0C39412900073F0800A90009D
:1045B90072E02412900073F0755D129000A7E0FE7E
:1045C9009000EDE0D39E50139000A7E0FE9000ED1F
:1045D900E0F4042E04900064F080139000A7E02416
:1045E90024FE9000EDE0F4042E04900064F09000A5
:1045F90064E075F00684AFF07E00EF4E700690001F
:1046090064E004F0900064E00475F00684AFF07E85
:1046190000EF4E7006900064E014F0900064E0B47E
:1046290025069000647401F0900064E0240690006F
:1046390065F0900064E0240C900066F0900064E05E
:104649002412900067F0900064E02418900068F04C
:10465900900064E0241E900069F0900065E0D39416
:1046690024400B900065E0C39424900065F090000D
:1046790066E0D39424400B900066E0C39424900034
:1046890066F0900067E0D39424400B900067E0C384
:104699009424900067F0900068E0D39424400B9034
:1046A9000068E0C39424900068F0900069E0D39416
:1046B90024400B900069E0C39424900069F0120132
:1046C9009C22C293C294C291C292C287C290E5B59C
:1046D90054EFF5B5E5B554DFF5B5C296C295C2A05C
:1046E900C297C2A2C2A1E5B554BFF5B5E5B5547FDD
:1046F900F5B5E5B554FBF5B5C208755E469000F011
:10470900E07005756D028003756D0375540075536E
:104719000090001874FFF0A374DCF0C20EC210C23E
:1047290012C214C216C21874C8900046F074C89018
:10473900004AF074C890004EF074C8900052F074AA
:10474900C8900056F074C890005AF075520075511F
:1047590000C203754600E56FB41303756F007563F6
:1047690000900026E4F0A3F0757010C20BC20CC2D1
:104779000DC20275560075550090001AE4F0A3F0B9
:1047890090001CE4F0A3F0C22475580075570090FE
:1047990000B2E075F032A4FFAEF090002EEEF0A367
:1047A900EFF0900910E4F022755A00755900AE59DE
:1047B900AF5A7422C39F74019E50030248A5906E9C
:1047C90086120048E493645F6023906E8612004865
:1047D900E493647E6017906E86120048E4936481C6
:1047E900600B906E86120048E493B48403024885F6
:1047F900AE59AF5A906E86120048E4939000A61203
:1048090071A30FBF00010EE0FC906E86120048EC08
:10481900FEE493FFEEC39F5026AE59AF5A0FBF0077
:10482900010E906E86120048AE59AF5AE493FC907F
:104839006E86120048E4939000A61271A3ECF0AEC4
:1048490059AF5A906E86120048E4939000A61271EF
:10485900A3E0FC906E88120048ECFCE493FDECD3D5
:104869009D4019906E88120048E493FC906E861260
:104879000048E4939000A61271A3ECF0AE59AF5A28
:1048890074022FFF50010E8E598F5A785A740126DF
:10489900F6500418E436F640030247B722755A0069
:1048A900755900AE59AF5A7432BE00039F500302C6
:1048B9004973906FA9120048E4939000A61271A35E
:1048C9000FBF00010EE0FC906FA9120048ECFEE456
:1048D90093FFEEC39F5026AE59AF5A0FBF00010E8A
:1048E900906FA9120048AE59AF5AE493FC906FA992
:1048F900120048E4939000A61271A3ECF0AE59AFF0
:104909005A906FA9120048E4939000A61271A3E08F
:10491900FC906FAB120048ECFCE493FDECD39D4096
:1049290019906FAB120048E493FC906FA9120048EC
:10493900E4939000A61271A3ECF0AE59AF5A742D0E
:104949006F4E7006755A33755900AE59AF5A7402D5
:104959002FFF50010E8E598F5A785A740126F6503E
:104969000418E436F640030248AC2275A71085F90D
:104979007385FA747E017F00E574127172E5732FF5
:10498900FF50010E8E598F5AAC5BAD5CEF2DFDEED9
:104999003CFC8C5B8D5CD293D294D291D292D2871B
:1049A900D290E55CF5FBE55BF5FCE55CF5E9E55BDB
:1049B900F5EAE55CF5EBE55BF5ECE55CF5EDE55B6A
:1049C900F5EEE55CF5FDE55BF5FEE55CF5CEE55B51
:1049D900F5CF75A7002285F97385FA747E017F00EA
:1049E900E574127172E5732FFF50010E8E598F5ABB
:1049F9007E017F7690012BE0127172AC59AD5AEDB0
:104A09002FFFEC3EFE8E5B8F5CE55CF5E9E55BF51F
:104A1900EA900098E4F07412900075F02285F97319
:104A290085FA747E017F00E574127172E5732FFFB8
:104A390050010E8E598F5A900020E0FCA3E0FDEF43
:104A49002DFDEE3CFC8C5B8D5CE55CF5FBE55BF5D7
:104A5900FC22056422A2D9B340089000FAE0900034
:104A690098F0A2D8B3400CC296C295C2A0C297C210
:104A7900A2C2A175D8402285A77275A710A2D8B382
:104A89004002C293A2D9B34002C294A2DAB340024F
:104A9900C291A2DBB34002C292A2DCB34002C28738
:104AA900A2DDB34002C29075D8408572A72290F862
:104AB90000E4936406600280FE12009E75A70075EB
:104AC900D80075D90475DA0975DB0975D84075A759
:104AD9001075D80075D90475DA0975DB0975DC0913
:104AE90075DD0975DE0975DF0975D84075A70012EE
:104AF90000FB74C8F5097508001205E475A70FE5F0
:104B0900FC900084F0E5FB900085F0E5FA900086C2
:104B1900F0E5F9900087F075A70090F800E493F5A7
:104B2900271207039008BDE0D3940350079008BDEE
:104B3900E0B4010674009008BDF09008BDE090094A
:104B490014F074019000EFF09008BDE0906A8AF8C3
:104B5900282873802A802875A70F75F30F75A70079
:104B6900A2A3400674029000EFF0801375A70F7599
:0F4B7900F31775A700A2A4400674029000EFF096
:0C6A8A00024B5C024B5E024B60024B753D
:104B88009000EFE0B4022AC21C120AAC7402900032
:104B9800EFF09008BDE0906A96F82828738010809E
:0F4BA8000E74009000FEF08006740090010BF078
:0C6A9600024BA5024BA7024BA9024BB11A
:104BB7008028D21C1209C174019000EFF09008BD43
:104BC700E0906AA2F82828738010800E7400900085
:0A4BD700FEF08006740090010BF060
:0C6AA200024BCF024BD1024BD3024BDB66
:104BE10090F807E493900091F0900091E0440890D0
:104BF1000091F0900091E054FE900091F012039D1D
:104C0100123DBA9008CAE0900192F09008CBE09072
:104C11000193F09008CCE0900194F0900192E07043
:104C21000C900193E07006900194E060028004C250
:104C3100218002D2219000E0E00490009CF09000DD
:104C4100D3E0049000A2F01247B11248A67400907C
:104C51000116F0123EF5E5B54401F5B57406900074
:104C610077F07400900078F07401900079F090F87A
:104C710002E49390007AF090F803E49390007BF0C3
:104C810090F804E49390007CF0740690007DF07439
:104C91003B90007EF0740390007FF07406900080DA
:104CA100F07407900081F090F805E493900082F091
:104CB10090F806E493900083F0740090008BF074F8
:104CC1000090008CF0740090008DF0740090008EC4
:104CD100F0740090008FF07400900090F074FF90D9
:104CE1000092F0A2B6B39204A2B3B39205A2A4B308
:104CF100921EA2A3B3921F900093E4F0756F00740B
:104D01003A9007A6F074FD9007A7F0900094E4F0A4
:104D1100756E01900075E4F09000F0E0B401067446
:104D21001A900075F0C21D756300C209D20AC20251
:104D3100757100C220120586755F00756B00756183
:104D410000756532756600756700756800756900E4
:104D5100756A00900026E4F0A3F0756C00D2B2D21F
:104D6100A4D2B0D2B1D2A3D2A7D2A6D2A5D2B77EB5
:104D7100017F009000CDE01271729000CCE02FFF16
:104D810050010E900030EEF0A3EFF0EFD394FFEE60
:104D9100940F4007900030E4F0A3F0900115E0700B
:104DA1000674FF900115F09000F0E07005756D023A
:104DB1008003756D037407900133F074089001341A
:104DC100F0742A900135F074299006ECF074159076
:104DD1000794F07416900795F07417900796F07485
:104DE10018900797F07419900798F0741A90079922
:104DF100F0740090079AF0740090079BF074019092
:104E0100079CF0740290079DF0740390079EF07464
:104E11000490079FF074059007A0F074069007A115
:104E2100F074009007A2F074009007A3F0D29CE503
:104E310070D3941040037570109006EDE0D3940C7C
:104E4100400674009006EDF09006F1E0D3940C401A
:104E51000674009006F1F09006F5E0D3940C40063C
:104E610074009006F5F09006F9E0D3940C400674B6
:104E7100009006F9F0D2EC75CF01A298B34005C2BB
:104E810098120C14E54D6006A299B3B34002800557
:104E9100C2991210A3E54E64016005E54EB4040207
:104EA10080D5C28E7E107F00E564127172E58D752A
:104EB100F010A4FDACF0EF2DFDEE3CFCE58B75F0A0
:104EC1001084FF7E00ED2FFFEC3EFE8E538F54D2F7
:104ED1008E9000D3E060099000D3E0C3943D40027E
:104EE1008056900028127180900028E0FEA3E0FF18
:104EF10090002AE0FCA3E0FDEFB5053CEEB50438D7
:104F0100B21AA203B34013A21AB34008E5B5440490
:104F1100F5B58006E5B554FBF5B590002AE0FEA392
:104F2100E0FF90002CE0FCA3E0FDEF2DFDEE3CFC4A
:104F310090002AECF0A3EDF09000E0E06009900011
:104F4100E0E0C3940340028077122FCEA203400811
:104F51009000CAE0F545801BE55FC395605005757B
:104F61004500800F9000B7E0C3956150069000DDC9
:104F7100E0F545E54575F002A4FFAEF09008B2EE0C
:104F8100F0A3EFF0AC2EAD2FEDD39FEC9E4015E5D5
:104F9100B554BFF5B59000E0E0B40206E5B5448034
:104FA100F5B5801C900093E0C3942E5013E5B544F1
:104FB10040F5B59000E0E0B40206E5B5547FF5B5E3
:104FC1009000E0E0B403241230E9AE2EAF2F900838
:104FD100B2E0FCA3E0FDEFD39DEE9C4008E5B544B3
:104FE10040F5B58006E5B554BFF5B5A2B63004016C
:104FF100B350030255CFA2B6300401B3500302559A
:10500100CFA2B6300601B350030254B1756E0090C1
:1050110000D3E0B43D13A206B34008E5B554FBF557
:10502100B58006E5B54404F5B5055EA208B3B350F5
:1050310013AE53AF54900018E0FCA3E0FDEDC39F05
:10504100EC9E4003025163E56DB4032EA224B340EC
:1050510022E55EB42303756D01E55EC3942350061A
:105061009000757401F0E55ED394234006740290BC
:105071000075F0755E01D2248062E56DB40206759B
:105081006D01755E23E55EB42305755E01804D906B
:105091000075E07038E55EC3942350069000757486
:1050A10001F0E55ED3942340067402900075F0E5AB
:1050B1005EC394235002D21DE55ED394234002D2F5
:1050C1001DC296C295C2A0C297C2A2C2A19000F011
:1050D100E0B401051246CB8003755E01AE55AF56B3
:1050E100AC53AD54EF2DFDEE3CFC74028C068D07E4
:1050F1001200398E558F569000D3E060099000D38D
:10510100E0C3943D40028043900028E0FEA3E0FF0D
:105111009000D3E08E048F05FF12716274018C063A
:105121008D0712003990002CEEF0A3EFF090002CC7
:10513100E0F8A3E090002AC8F0A3C8F0900028E4AA
:10514100F0A3F0C21AE5B554FBF5B5A2A4B3400231
:10515100C21EA2A3B34002C21FA21DB34002C21DC0
:10516100803AAE55AF56AC53AD54EF2DFDEE3CFC3D
:1051710074018C068D071200398E558F56E56DC36B
:105181009402500DAC53AD547488C39D74139C406C
:105191000280091246CB7406900075F0E55EB423D7
:1051A100127403900075F0D21D9000F0E0B4010379
:1051B1001246CBAE57AF58AC53AD54EF2DFDEE3C7C
:1051C100FC8C578D58AE53AF54EFD39DEE9C4011DC
:1051D10090001EE0FAA3E0FBEBC394E8EA940340DD
:1051E10002800690001E12718090001CE0FEA3E078
:1051F100FFAC53AD54EF2DFDEE3CFC90001CECF0E8
:10520100A3EDF09000F0E0B40118AE53AF54740573
:105211001271727401120039900018EEF0A3EFF0D0
:105221008011AE53AF547402127172900018EEF0F7
:10523100A3EFF0C28E758D00758B007564007554F7
:1052410001755300D28EE55E240875F00984AFF034
:105251007E00EF4E60030252DCE56D6013AE55AF88
:1052610056740912717290001AEEF0A3EFF0800FDC
:1052710090001CE0F8A3E090001AC8F0A3C8F090D9
:10528100001AE0FEA3E0FFEF4E600B7C837D9012DD
:1052910070608E518F5290001CE4F0A3F0AE51AFBC
:1052A100527428BE00039F5010E5632FFF50010E7A
:1052B10074011200398E518F528552639000F7E0CC
:1052C100A851B8000DD395524008E552900074F0F2
:1052D10080099000F7E014900074F0E55E640B60C3
:1052E10005E55EB41D099000E0E06003122C849096
:1052F1000072E0655E6007900073E0B55E03756F54
:1053010000A209B35006A208B3B340030253B590FB
:1053110000ACE0B4017390012EE0B4021412124407
:10532100900099E075F0BCA4FFAEF08E5B8F5C80BD
:1053310056E56775F00A84FF7E009005A6120048C5
:10534100E0F55A755900AE59AF5A9000D1E012718B
:105351007274648E048F05FF1271628C5B8D5CE543
:105361005C900070F0AE59AF5A9000AAE0127172D1
:1053710074648E048F05FF12716274BC8C068D07F4
:105381001271728E5B8F5C80179000AAE075F0BC81
:10539100A4FFAEF08E5B8F5C9000D1E0900070F0C6
:1053A100E561C394CC5006E55C455B700280031255
:1053B1004974D209E56DB40106E55E640B600280B3
:1053C1000C7570009000767401F0756D00E56D60EC
:1053D100030254AC9000F3E0600D900098E0A851F6
:1053E100B800069552400280589000F3E0B40237AD
:1053F10090005EE0655E602790005FE0655E601F83
:10540100900060E0655E6017900061E0655E600F8E
:10541100900062E0655E6007900063E0B55E037531
:105421007003756C00800CC200756C00900026E45E
:10543100F0A3F0900098E060067409900075F08088
:105441006A90005EE0B55E0B7570009000767401A5
:10545100F0805890005FE0B55E0B757000740290AB
:105461000076F08046900060E0B55E0B75700074C8
:1054710003900076F08034900061E0B55E0B7570AA
:10548100007404900076F08022900062E0B55E0B1B
:105491007570007405900076F08010900063E0B59F
:1054A1005E097570007406900076F0A206B392044E
:1054B100A206B330B601B350030255CF756E019009
:1054C10000D3E0B43D13A206B34008E5B54404F5AA
:1054D100B58006E5B554FBF5B5E5B54401F5B57400
:1054E1001F900093F0A2069204E55ED3944A401403
:1054F100D208E55ED3946D400B7405900075F0D22F
:105501001D755E46900129E0A851B80005D395525A
:10551100500D900128E0A851B80004955250028026
:1055210008E5B54402F5B5801790012AE0D39561ED
:105531004008E5B54402F5B58006E5B554FDF5B57D
:105541009000FBE0B40107E56AC394414002801872
:10555100E56AC3941450087413900075F0800674C2
:105561000E900075F01246CB90007DE0FE90007A1F
:10557100E0C39E400990007AE0D39408400974FB8F
:10558100900075F01246CB90007BE0601590007B97
:10559100E0FE900079E06E600974FC900075F012F5
:1055A10046CB90007CE0601590007CE0FE90007E90
:1055B100E06E600974FE900075F01246CB9008BD54
:1055C100E0600690012BE060028003120B97A21DA0
:1055D100B3400CC296C295C2A0C297C2A2C2A1900A
:1055E100012BE0600CAE51AF527414BE00059F4018
:1055F1000280379000B3E0906AAEF8282873802AC1
:105601008028A2A3B35005A21FB34002800512490E
:10561100DFD21F8015A2A4B35005A21EB3400280A1
:0A562100051249DFD21E800280004E
:106AAE000255FF02560102560302561602562902DD
:026ABE00562B55
:10562B00A20BB3B35008900064E0655E6002803655
:10563B00A201B35006A200B3B340028023123CD8A0
:10564B00123D1A90010CE0B40113A202B34008E51D
:10565B00B54480F5B58006E5B5547FF5B575A70063
:10566B00C20BD20CD20DA20CB3B35008900065E064
:10567B00655E60028036A201B35006A200B3B34050
:10568B00028023123CD8123D2590010CE0B401138B
:10569B00A202B34008E5B54480F5B58006E5B554E4
:1056AB007FF5B575A700D20BC20CD20DA20DB3B30B
:1056BB005008900066E0655E60028036A201B35030
:1056CB0006A200B3B340028023123CD8123D3090A7
:1056DB00010CE0B40113A202B34008E5B54480F518
:1056EB00B58006E5B5547FF5B575A700D20BD20C86
:1056FB00C20DA20BB3B35008900067E0655E600269
:10570B008036A201B35006A200B3B340028023122D
:10571B003CD8123D3B90010CE0B40113A202B34004
:10572B0008E5B54480F5B58006E5B5547FF5B5754C
:10573B00A700C20BD20CD20DA20CB3B35008900031
:10574B0068E0655E60028036A201B35006A200B32A
:10575B00B340028023123CD8123D4690010CE0B4BA
:10576B000113A202B34008E5B54480F5B58006E508
:10577B00B5547FF5B575A700D20BC20CD20DA20D97
:10578B00B3B35008900069E0655E60028036A201F9
:10579B00B35006A200B3B340028023123CD8123D93
:1057AB005190010CE0B40113A202B34008E5B544DB
:1057BB0080F5B58006E5B5547FF5B575A700D20B1E
:1057CB00D20CC20DE570906AC0F8282873900113B3
:0157DB00E0ED
:036AC0000257D8A2
:1057DC00906AF3F82828731225CF80121225CF80F7
:0E57EC000D122659800812270580031227058A
:0F6AF3000257E30257E80257ED0257F20257F736
:1057FA00757001025EAC12283112294875700202D6
:10580A005EAC122CC8A203B340139000F8E075F006
:10581A001DA4FFAEF0900020EEF0A3EFF09008A6D2
:10582A00E0FEA3E0FF740A12717290001AE0FCA372
:10583A00E0FD74098F02FF1271628D078C038E04DA
:10584A008A058B061270609008AAEEF0A3EFF07436
:10585A00F0BE00039F500B74F09008AAF8E4F0E839
:10586A00A3F0E53670037536019008AAE0FEA3E0BE
:10587A00FFE5362FFF50010E9008AAEEF0A3EFF0D5
:0B588A00757003A22B4029900076E00F
:066AC30002580002580C0D
:10589500906B02F8282873801C75700A8017757044
:1058A5000B801275700C800D75700D800875700E6B
:0558B500800375700F77
:106B020002589C02589E0258A30258A80258AD028D
:056B120058B20258B763
:1058BA00025EAC9006EDE060077401F508122DF661
:1058CA00A22DB3B350089007A4E0642960028009AE
:1058DA00E5B54408F5B50259849000E1E0D3940295
:1058EA0040459000B5E02403A851B80004955250F1
:1058FA00099000B7E0D395615002800ED201A2232D
:10590A0040067408900075F0D2239000B5E0A851C3
:10591A00B80005D39552500B9000B7E02403C39505
:10592A00615002C20180539000B5E02403A851B827
:10593A00000495525010E55FC3956050099000B776
:10594A00E0D395615002800ED201A223400674086A
:10595A00900075F0D2239000B5E0A851B80005D3A5
:10596A0095525014E560240FC3955F400B9000B721
:10597A00E02403C395615002C201A2014002C2237E
:10598A00A22DB3500DA201B350089007A4E06429D8
:10599A0060028006E5B554F7F5B59000FBE07007A4
:1059AA00E56AC3941440028002D2019000F0E0B488
:1059BA000102D201A2014005757004800A757010B7
:0E59CA00900026E4F0A3F0025EAC9000E1E055
:066AC9000258BD0259D481
:1059D800906B17F828287312135A801212135A80E2
:0E59E8000D12150D80081215C480031215C48F
:0F6B17000259DF0259E40259E90259EE0259F31B
:1059F6009006F1E060077402F508122DF675700541
:105A0600025EAC12171D7570069006F5E06007740D
:105A160003F508122DF6025EAC900070E06006A257
:105A260003B3B34002800DE55ED3940650069000A2
:105A360070E014F01219A67570079006F9E0600779
:105A46007404F508122DF6025EAC90012EE0B40245
:105A5600031212CB121E0E757008025EAC121EF0F7
:105A6600757009025EAC1222C8A20BB35005A20CD7
:105A7600B340028006D20BD20CD20D757010025EB6
:105A8600AC900048E0C394465008C2967446900015
:105A960048F090006AE0B4011DE536240AF5369018
:105AA60008AAE0FEA3E0FF740A2FFF50010E90083B
:105AB600AAEEF0A3EFF090006AE0B4021DE53624EA
:105AC60014F5369008AAE0FEA3E0FF74142FFF50E9
:105AD600010E9008AAEEF0A3EFF085365A7559002C
:105AE60090005EE0F573123E5EE55C900048F09033
:105AF600000CE559F0A3E55AF0E573900049F0C2B1
:105B06000F9008AAE0F559A3E0F55A90005EE0F57B
:105B160073123E5EE55C900046F0900000E559F099
:105B2600A3E55AF0E573900047F0C20E75700302C4
:105B36005EAC90004CE0C394465008C29574469003
:105B4600004CF090006BE0B4011DE536240AF536F2
:105B56009008AAE0FEA3E0FF740A2FFF50010E9002
:105B660008AAEEF0A3EFF090006BE0B4021DE53654
:105B76002414F5369008AAE0FEA3E0FF74142FFF64
:105B860050010E9008AAEEF0A3EFF085365A75592B
:105B96000090005FE0F573123E5EE55C90004CF00D
:105BA60090000EE559F0A3E55AF0E57390004DF02C
:105BB600C2119008AAE0F559A3E0F55A90005FE0FB
:105BC600F573123E5EE55C90004AF0900002E559DE
:105BD600F0A3E55AF0E57390004BF0C21075700320
:105BE600025EAC900050E0C394465008C2A07446D2
:105BF600900050F090006CE0B4011DE536240AF5E3
:105C0600369008AAE0FEA3E0FF740A2FFF50010EAB
:105C16009008AAEEF0A3EFF090006CE0B4021DE548
:105C2600362414F5369008AAE0FEA3E0FF74142F7C
:105C3600FF50010E9008AAEEF0A3EFF085365A75D4
:105C46005900900060E0F573123E5EE55C900050EE
:105C5600F0900010E559F0A3E55AF0E57390005175
:105C6600F0C2139008AAE0F559A3E0F55A90006037
:105C7600E0F573123E5EE55C90004EF0900004E5A0
:105C860059F0A3E55AF0E57390004FF0C212757013
:105C960003025EAC900054E0C394465008C2977469
:105CA60046900054F090006DE0B4011DE536240ADC
:105CB600F5369008AAE0FEA3E0FF740A2FFF500114
:105CC6000E9008AAEEF0A3EFF090006DE0B4021D6E
:105CD600E5362414F5369008AAE0FEA3E0FF741416
:105CE6002FFF50010E9008AAEEF0A3EFF085365A6A
:105CF600755900900061E0F573123E5EE55C900018
:105D060054F0900012E559F0A3E55AF0E5739000BF
:105D160055F0C2159008AAE0F559A3E0F55A90008F
:105D260061E0F573123E5EE55C900052F09000066D
:105D3600E559F0A3E55AF0E573900053F0C21475E7
:105D46007003025EAC900058E0C394465008C2A2AD
:105D56007446900058F090006EE0B4011DE53624BC
:105D66000AF5369008AAE0FEA3E0FF740A2FFF505A
:105D7600010E9008AAEEF0A3EFF090006EE0B402D8
:105D86001DE5362414F5369008AAE0FEA3E0FF745C
:105D9600142FFF50010E9008AAEEF0A3EFF08536FF
:105DA6005A755900900062E0F573123E5EE55C900C
:105DB6000058F0900014E559F0A3E55AF0E5739009
:105DC6000059F0C2179008AAE0F559A3E0F55A90D9
:105DD6000062E0F573123E5EE55C900056F09000BE
:105DE60008E559F0A3E55AF0E573900057F0C2169E
:105DF600757003025EAC90005CE0C394465008C226
:105E0600A1744690005CF090006FE0B4011DE53689
:105E1600240AF5369008AAE0FEA3E0FF740A2FFFD5
:105E260050010E9008AAEEF0A3EFF090006FE0B4D8
:105E3600021DE5362414F5369008AAE0FEA3E0FF1D
:105E460074142FFF50010E9008AAEEF0A3EFF08510
:105E5600365A755900900063E0F573123E5EE55CB4
:105E660090005CF0900016E559F0A3E55AF0E57352
:105E760090005DF0C2199008AAE0F559A3E0F55A22
:105E8600900063E0F573123E5EE55C90005AF09078
:105E9600000AE559F0A3E55AF0E57390005BF0C2FD
:065EA60018757003800076
:106ACF00025A09025A1F025A50025A63025A6C02A2
:106ADF005A87025B38025BE9025C9A025D4B025DEA
:046AEF00FC025EAC9B
:105EAC00900046E0B55E028003025F4EA20E407287
:105EBC00900000E0FEA3E0FFEF4E6021AE55AF5620
:105ECC00900000E0FCA3E0FD120003740A8E048F26
:105EDC0005FF127162900000ECF0A3EDF09000470A
:105EEC00E0601A900000E0FEA3E0FFAC55AD56EF69
:105EFC002DFDEE3CFC900000ECF0A3EDF090004783
:105F0C00E0D39401401A900000E0FEA3E0FFAC55F2
:105F1C00AD56EF2DFDEE3CFC900000ECF0A3EDF047
:105F2C00D20EAE53AF54900000E0FCA3E0FDEFC3E3
:105F3C009DEE9C400D124A26D296C20E74C890005B
:105F4C0046F0A20EB3B35007900046E0B55E028057
:105F5C000D124A26D29674C8900046F0C20E9000DC
:105F6C0048E0B55E028003026009A20F4072900007
:105F7C000CE0FEA3E0FFEF4E6021AE55AF56900053
:105F8C000CE0FCA3E0FD120003740A8E048F05FFE5
:105F9C0012716290000CECF0A3EDF0900049E060FF
:105FAC001A90000CE0FEA3E0FFAC55AD56EF2DFDB2
:105FBC00EE3CFC90000CECF0A3EDF0900049E0D32B
:105FCC009401401A90000CE0FEA3E0FFAC55AD56D6
:105FDC00EF2DFDEE3CFC90000CECF0A3EDF0D20F9D
:105FEC00AE53AF5490000CE0FCA3E0FDEFC39DEE6C
:105FFC009C400AC2967446900048F0C20FA20FB3A0
:10600C00B35007900048E0B55E02800AC296744611
:10601C00900048F0C20F90004AE0B55E0280030287
:10602C0060C4A2104072900002E0FEA3E0FFEF4EAD
:10603C006021AE55AF56900002E0FCA3E0FD1200CB
:10604C0003740A8E048F05FF127162900002ECF04B
:10605C00A3EDF090004BE0601A900002E0FEA3E08C
:10606C00FFAC55AD56EF2DFDEE3CFC900002ECF074
:10607C00A3EDF090004BE0D39401401A900002E0A5
:10608C00FEA3E0FFAC55AD56EF2DFDEE3CFC9000B1
:10609C0002ECF0A3EDF0D210AE53AF54900002E03E
:1060AC00FCA3E0FDEFC39DEE9C400D124A26D29559
:1060BC00C21074C890004AF0A210B3B350079000FD
:1060CC004AE0B55E02800D124A26D29574C8900043
:1060DC004AF0C21090004CE0B55E02800302617F72
:1060EC00A211407290000EE0FEA3E0FFEF4E602183
:1060FC00AE55AF5690000EE0FCA3E0FD1200037409
:10610C000A8E048F05FF12716290000EECF0A3ED65
:10611C00F090004DE0601A90000EE0FEA3E0FFACA2
:10612C0055AD56EF2DFDEE3CFC90000EECF0A3EDC2
:10613C00F090004DE0D39401401A90000EE0FEA3C5
:10614C00E0FFAC55AD56EF2DFDEE3CFC90000EEC97
:10615C00F0A3EDF0D211AE53AF5490000EE0FCA3BF
:10616C00E0FDEFC39DEE9C400AC295744690004C36
:10617C00F0C211A211B3B3500790004CE0B55E020F
:10618C00800AC295744690004CF0C21190004EE00B
:10619C00B55E02800302623AA2124072900004E0E3
:1061AC00FEA3E0FFEF4E6021AE55AF56900004E029
:1061BC00FCA3E0FD120003740A8E048F05FF12711C
:1061CC0062900004ECF0A3EDF090004FE0601A90A8
:1061DC000004E0FEA3E0FFAC55AD56EF2DFDEE3C08
:1061EC00FC900004ECF0A3EDF090004FE0D3940190
:1061FC00401A900004E0FEA3E0FFAC55AD56EF2D25
:10620C00FDEE3CFC900004ECF0A3EDF0D212AE538A
:10621C00AF54900004E0FCA3E0FDEFC39DEE9C4066
:10622C000D124A26D2A0C21274C890004EF0A212CF
:10623C00B3B3500790004EE0B55E02800D124A26B3
:10624C00D2A074C890004EF0C212900050E0B55E1F
:10625C000280030262F5A2134072900010E0FEA3CC
:10626C00E0FFEF4E6021AE55AF56900010E0FCA35E
:10627C00E0FD120003740A8E048F05FF1271629008
:10628C000010ECF0A3EDF0900051E0601A900010BB
:10629C00E0FEA3E0FFAC55AD56EF2DFDEE3CFC90BF
:1062AC000010ECF0A3EDF0900051E0D39401401AF3
:1062BC00900010E0FEA3E0FFAC55AD56EF2DFDEEC7
:1062CC003CFC900010ECF0A3EDF0D213AE53AF54A5
:1062DC00900010E0FCA3E0FDEFC39DEE9C400AC2D1
:1062EC00A07446900050F0C213A213B3B3500790A1
:1062FC000050E0B55E02800AC2A07446900050F0D7
:10630C00C213900052E0B55E0280030263B0A21487
:10631C004072900006E0FEA3E0FFEF4E6021AE5508
:10632C00AF56900006E0FCA3E0FD120003740A8E49
:10633C00048F05FF127162900006ECF0A3EDF09053
:10634C000053E0601A900006E0FEA3E0FFAC55ADF0
:10635C0056EF2DFDEE3CFC900006ECF0A3EDF0901A
:10636C000053E0D39401401A900006E0FEA3E0FF36
:10637C00AC55AD56EF2DFDEE3CFC900006ECF0A3B9
:10638C00EDF0D214AE53AF54900006E0FCA3E0FD48
:10639C00EFC39DEE9C400D124A26D297C21474C8CE
:1063AC00900052F0A214B3B35007900052E0B55EC7
:1063BC0002800D124A26D29774C8900052F0C21473
:1063CC00900054E0B55E02800302646BA21540722B
:1063DC00900012E0FEA3E0FFEF4E6021AE55AF56E9
:1063EC00900012E0FCA3E0FD120003740A8E048FEF
:1063FC0005FF127162900012ECF0A3EDF0900055C5
:10640C00E0601A900012E0FEA3E0FFAC55AD56EF31
:10641C002DFDEE3CFC900012ECF0A3EDF09000553D
:10642C00E0D39401401A900012E0FEA3E0FFAC55BB
:10643C00AD56EF2DFDEE3CFC900012ECF0A3EDF010
:10644C00D215AE53AF54900012E0FCA3E0FDEFC3A5
:10645C009DEE9C400AC2977446900054F0C215A25F
:10646C0015B3B35007900054E0B55E02800AC29792
:10647C007446900054F0C215900056E0B55E028050
:10648C0003026526A2164072900008E0FEA3E0FF0E
:10649C00EF4E6021AE55AF56900008E0FCA3E0FD36
:1064AC00120003740A8E048F05FF127162900008AB
:1064BC00ECF0A3EDF0900057E0601A900008E0FEBD
:1064CC00A3E0FFAC55AD56EF2DFDEE3CFC90000863
:1064DC00ECF0A3EDF0900057E0D39401401A90003B
:1064EC0008E0FEA3E0FFAC55AD56EF2DFDEE3CFCF5
:1064FC00900008ECF0A3EDF0D216AE53AF54900020
:10650C0008E0FCA3E0FDEFC39DEE9C400D124A2673
:10651C00D2A2C21674C8900056F0A216B3B350079C
:10652C00900056E0B55E02800D124A26D2A274C8C5
:10653C00900056F0C216900058E0B55E028003023F
:10654C0065E1A2174072900014E0FEA3E0FFEF4E4D
:10655C006021AE55AF56900014E0FCA3E0FD120094
:10656C0003740A8E048F05FF127162900014ECF014
:10657C00A3EDF0900059E0601A900014E0FEA3E047
:10658C00FFAC55AD56EF2DFDEE3CFC900014ECF03D
:10659C00A3EDF0900059E0D39401401A900014E060
:1065AC00FEA3E0FFAC55AD56EF2DFDEE3CFC90008C
:1065BC0014ECF0A3EDF0D217AE53AF54900014E0EE
:1065CC00FCA3E0FDEFC39DEE9C400AC2A274469072
:1065DC000058F0C217A217B3B35007900058E0B59B
:1065EC005E02800AC2A27446900058F0C217900056
:1065FC005AE0B55E02800302669CA21840729000BD
:10660C000AE0FEA3E0FFEF4E6021AE55AF569000BE
:10661C000AE0FCA3E0FD120003740A8E048F05FF50
:10662C0012716290000AECF0A3EDF090005BE06058
:10663C001A90000AE0FEA3E0FFAC55AD56EF2DFD1D
:10664C00EE3CFC90000AECF0A3EDF090005BE0D384
:10665C009401401A90000AE0FEA3E0FFAC55AD5641
:10666C00EF2DFDEE3CFC90000AECF0A3EDF0D218FF
:10667C00AE53AF5490000AE0FCA3E0FDEFC39DEED7
:10668C009C400D124A26D2A1C21874C890005AF030
:10669C00A218B3B3500790005AE0B55E02800D12F9
:1066AC004A26D2A174C890005AF0C21890005CE03F
:1066BC00B55E028003026757A2194072900016E083
:1066CC00FEA3E0FFEF4E6021AE55AF56900016E0F2
:1066DC00FCA3E0FD120003740A8E048F05FF1271F7
:1066EC0062900016ECF0A3EDF090005DE0601A9063
:1066FC000016E0FEA3E0FFAC55AD56EF2DFDEE3CD1
:10670C00FC900016ECF0A3EDF090005DE0D394014A
:10671C00401A900016E0FEA3E0FFAC55AD56EF2DED
:10672C00FDEE3CFC900016ECF0A3EDF0D219AE534C
:10673C00AF54900016E0FCA3E0FDEFC39DEE9C402F
:10674C000AC2A1744690005CF0C219A219B3B350EE
:10675C000790005CE0B55E02800AC2A1744690000E
:10676C005CF0C2199000FEE0B4020280030268984B
:10677C00900095E0D395665064900095E0F4042564
:10678C0066FE900101E08E00F5F0E884FF7E008F3C
:10679C0073EFC39410500CEF8573F0A4FDACF08D27
:1067AC007380037573FF900095E0D39573400B9045
:1067BC000095E0C39573F571800375710090011C11
:1067CC00E0D39571400690011CE0F57190011DE03D
:1067DC00C39571500690011DE0F571807190009584
:1067EC00E0C39566FE900101E08E00F5F0E884FFB1
:1067FC007E008F73EFC39410500CEF8573F0A4FDE3
:10680C00ACF08D7380037573FF85735A75590090C6
:10681C000095E0255AFFAE5950010E8E598F5A74CF
:10682C00FFBE0009D39F4005855A7180037571FF27
:10683C0090011CE0D39571400690011CE0F571901D
:10684C00011DE0C39571500690011DE0F571A20386
:10685C00B3B3500D900096E0FE900109E0D39E502A
:10686C0002800E7407900075F0E5B554BFF5B58045
:10687C001B75A710E5CDC395714008E5B554BFF560
:10688C00B58006E5B54440F5B575A700900123E049
:10689C00A851B80005D395525016900122E0A8518A
:1068AC00B8000D95524009900124E0D39561400247
:1068BC00802975A710E5CDC394BF400EE5B554EF04
:1068CC00F5B5E5B554DFF5B5800CE5B54410F5B577
:1068DC00E5B54420F5B575A700802775A710E5CD63
:1068EC00C39440400EE5B554EFF5B5E5B554DFF56E
:1068FC00B5800CE5B54410F5B5E5B54420F5B57596
:10690C00A700E56FC39413501DE56F75F00284AFBB
:10691C00F07E00EF4E7005123290800AA2EDB3406B
:10692C0005C2ED123290AE53AF547498C39F743AB3
:10693C009E400C900094E0C3945A4003026A78A2E3
:10694C0008B340091246CB7406900075F0A20AB346
:10695C00500EE561D394334007E561C394CC4002FB
:10696C00804190012EE0B40214121244900099E080
:10697C0075F05EA4FFAEF08E5B8F5C800F9000AA6A
:10698C00E075F05EA4FFAEF08E5B8F5CE55C455B62
:10699C006011E5B54401F5B5741F900093F01249F0
:1069AC0074D20A900094E0D394014007E561C3943B
:1069BC001A40028002C20A9006EDE060077401F5ED
:1069CC0008122DF69006F1E060077402F508122DFE
:1069DC00F69006F5E060077403F508122DF69006A4
:1069EC00F9E060077404F508122DF6900094E0C3EA
:1069FC00945A5010E56FB41309900094E004F075AC
:106A0C006F00803FE56FB41303756F00C28E758DF8
:106A1C0000758B00756400755401755300D28E900F
:106A2C000093E0C3942E5008900093E004F080068D
:106A3C00742E900093F0900093E0B42E06E5B554BC
:106A4C00FEF5B5900094E0D394014007E56AC39439
:106A5C004140028006740E900075F09008BDE06015
:0F6A6C000690012BE060028003120B97024E7818
:106B26000000010001400160018001A001C001E0F8
:106B360002000300039603B603D603F4040005001F
:106B46000512052405360548055A056C057E05908F
:106B560005A805C005DE0600061406280646066ECC
:106B660006AE05CF06EE00FF013F015F017F019FE4
:106B760001BF01DF01FF02FF039503B503D503F350
:106B860003FF04FF05110523053505470559056B68
:106B9600057D058F05A705BF05CE05F1061306275A
:106BA6000645066D06AD06ED05DD06FF0FAA0FA527
:106BB6000F9F0F9A0F940F8D0F870F800F780F710D
:106BC6000F680F600F570F4E0F450F3B0F300F2505
:106BD6000F1A0F0E0F020EF50EE80EDB0ECC0EBED0
:106BE6000EAE0E9F0E8E0E7D0E6C0E5A0E470E3496
:106BF6000E200E0C0DF70DE20DCB0DB50D9D0D857E
:106C06000D6D0D540D3A0D200D050CE90CCE0CB191
:106C16000C940C760C580C3A0C1B0BFB0BDB0BBBC9
:106C26000B9A0B790B570B350B130AF10ACE0AABED
:106C36000A870A640A400A1C09F809D409B0098CB3
:106C460009670943091F08FB08D608B2088E086AB7
:106C56000846082307FF07DC07B90796077307519D
:106C6600072F070D06EC06CA06AA06890669064915
:106C7600062A060A05EC05CD05B0059205750558E8
:106C8600053C0520050504EA04CF04B5049C0482EE
:106C96000469045104390422040B03F403DE03C817
:106CA60003B2039D038903750361034D033B032868
:106CB6000316030402F202E102D102C002B002A0EE
:106CC600029102820273026502570249023C022FB8
:106CD60002220216020901FD01F201E601DB01D0E2
:106CE60001C601BB01B101A7019D0194018B01827F
:106CF60001790170016801600158015001480141A4
:106D060001390132012B0125011E01180111010B68
:106D1600010500FF00FA0FA60FA00F990F920F8B27
:106D26000F840F7C0F740F6B0F620F580F4E0F43BB
:106D36000F380F2C0F1F0F120F050EF70EE80ED887
:106D46000EC80EB70EA50E930E800E6C0E580E4290
:106D56000E2C0E150DFD0DE40DCB0DB10D950D7917
:106D66000D5D0D3F0D200D010CE10CC00C9E0C7C41
:106D76000C590C350C100BEA0BC40B9E0B760B4F03
:106D86000B260AFD0AD40AAA0A800A550A2A09FF0E
:106D960009D409A8097C0950092508F908CD08A1D4
:106DA6000875084A081E07F307C8079D07730749B1
:106DB600072006F706CE06A6067E06570630060A02
:106DC60005E405BF059B057705540532051004EF5C
:106DD60004CE04AE048F047104530435041903FD74
:106DE60003E203C703AD0394037B0363034B03343E
:106DF600031E030802F302DE02CA02B602A30291D0
:106E0600027F026D025C024C023C022C021D020E45
:106E1600020001F201E401D701CA01BE01B101A6D7
:106E2600019A018F0185017A01700166015D0153A6
:106E3600014A0141013901310129012101190112DA
:106E4600010B010400FD00F700F000EA00E400DE9B
:106E560000D900D300CE00C900C400BF00BA00B5F7
:106E660000B100AD00A800A400A0009C0099009508
:106E76000091008E008A008700840081007E007BDE
:10009E0075B50075840175A70075FFA075EF069004
:1000AE000071E4F075C91075A70F75A1C775A7008B
:1000BE0075D90075CE0C75A70F75F1FE75F2FF752B
:1000CE00F30775F47875A4BA75A5FF75A60775AE16
:1000DE000075AFFF75D48175D5FF75D6FF75D7FF47
:1000EE0075A70075A20175A14775F8092275E60876
:1000FE0075E71075BC0175BE0475BD6C75BE0775D0
:10010E00BDA075BE0875BD0175BC0075BB1875BC6C
:10011E002075BA0875E88075D11375A70F75E105BE
:10012E0075E20075C7401246CB75970075978074BF
:10013E000A1271527597C0E5975420700280F875B7
:10014E008F0275A700D2AF75980075A90C75A70F11
:10015E0075AB4375ADFB75AC1E75A71075C91875DB
:10016E00CA0075CB0075C80475A700758912758E07
:10017E0004758C00758A00C2A9D28C758D00758BA2
:10018E0000D2ABD28E75B62075D944C2992290009A
:10019E00A8E09008BCF09000B3E09008BDF090008D
:1001AE00B4E09008BEF09000D3E09008BFF090004D
:1001BE00E0E09008C0F09000EEE09008C1F09000F2
:1001CE00FCE09008C2F09000FEE09008C3F09001B1
:1001DE000CE09008C4F0900119E09008C5F0900171
:1001EE001AE09008C6F090012CE09008C7F090013C
:1001FE0044E09008C9F0900192E09008CAF0900196
:10020E0093E09008CBF0900194E09008CCF0900130
:10021E002BE09008CDF0900115E09008CEF0900004
:10022E00CCE09008CFF09000CDE09008D0F0900098
:10023E00C7E09008D1F09000C8E09008D2F090018D
:10024E0031E09008D3F0900132E09008D4F09001A4
:10025E0033E09008D5F0900134E09008D6F090018C
:10026E0035E09008D7F09006ECE09008D8F09006B4
:10027E00F0E09008D9F09006F4E09008DAF09006DD
:10028E00F8E09008DBF09006FCE09008DCF09007B8
:10029E0000E09008DDF0900704E09008DEF0900793
:1002AE0008E09008DFF090070CE09008E0F090076F
:1002BE0010E09008E1F0900794E09008E2F09007CB
:1002CE0095E09008E3F0900796E09008E4F0900730
:1002DE0097E09008E5F0900798E09008E6F0900718
:1002EE0099E09008E7F090079AE09008E8F0900700
:1002FE009BE09008E9F090079CE09008EAF09007E8
:10030E009DE09008EBF090079EE09008ECF09007CF
:10031E009FE09008EDF09007A0E09008EEF09007B7
:10032E00A1E09008EFF09007A2E09008F0F090079F
:10033E00A3E09008F1F09007A4E09008F2F090018D
:10034E0036E09008F3F0900137E09008F4F0900159
:10035E0038E09008F5F0900139E09008F6F0900141
:10036E003AE09008F7F090013BE09008F8F0900129
:10037E003CE09008F9F090013DE09008FAF0900111
:10038E003EE09008FBF090013FE09008FCF02290D8
:10039E0008BCE09000A8F09008BDE09000B3F0908B
:1003AE0008BEE09000B4F09008BFE09000D3F0904B
:1003BE0008C0E09000E0F09008C1E09000EEF090F0
:1003CE0008C2E09000FCF09008C3E09000FEF090B0
:1003DE0008C4E090010CF09008C5E0900119F0906F
:1003EE0008C6E090011AF09008C7E090012CF0903A
:1003FE0008C9E0900144F09008CDE090012BF090F8
:10040E0008CEE0900115F09008CFE09000CCF0906F
:10041E0008D0E09000CDF09008D1E09000C7F090A9
:10042E0008D2E09000C8F09008D3E0900131F0902F
:10043E0008D4E0900132F09008D5E0900133F090AE
:10044E0008D6E0900134F09008D7E0900135F09096
:10045E0008D8E09006ECF09008D9E09006F0F09005
:10046E0008DAE09006F4F09008DBE09006F8F090E1
:10047E0008DCE09006FCF09008DDE0900700F090BC
:10048E0008DEE0900704F09008DFE0900708F09097
:10049E0008E0E090070CF09008E1E0900710F09073
:1004AE0008E2E0900794F09008E3E0900795F09052
:1004BE0008E4E0900796F09008E5E0900797F0903A
:1004CE0008E6E0900798F09008E7E0900799F09022
:1004DE0008E8E090079AF09008E9E090079BF0900A
:1004EE0008EAE090079CF09008EBE090079DF090F2
:1004FE0008ECE090079EF09008EDE090079FF090DA
:10050E0008EEE09007A0F09008EFE09007A1F090C1
:10051E0008F0E09007A2F09008F1E09007A3F090A9
:10052E0008F2E09007A4F09008F3E0900136F09006
:10053E0008F4E0900137F09008F5E0900138F09063
:10054E0008F6E0900139F09008F7E090013AF0904B
:10055E0008F8E090013BF09008F9E090013CF09033
:10056E0008FAE090013DF09008FBE090013EF0901B
:10057E0008FCE090013FF0227547009008B4E4F0CB
:10058E00A3F0753100753000754D00754E00C22711
:10059E00D2289008BDE06002D22074FE9008B6F812
:1005AE00E4F0E8A3F074FE9008BAF8E4F0E8A3F0E3
:1005BE0074FE9008B8F8E4F0E8A3F0745A90090EAF
:1005CE00F0745A90090FF0D229C225C22BC22AC24A
:1005DE0026C22DC23322750B00750A00AE0AAF0B70
:1005EE00AC08AD09EDC39FEC9E401674FF1271521C
:1005FE0075CF01780B740126F6500418E436F650C8
:10060E00DB22C2AF75D904758F0375B7A575B7F127
:10061E0090F800E4F0758F0175B7A575B7F1E52771
:10062E0090F800F075B7A575B7F190F801E4F07584
:10063E00B7A575B7F1900902E090F802F075B7A56D
:10064E0075B7F1900906E090F803F075B7A575B788
:10065E00F1900903E090F804F075B7A575B7F19025
:10066E000904E090F805F075B7A575B7F190090586
:10067E00E090F806F075B7A575B7F1900907E09010
:10068E00F807F0758F0075D944D2AF22900071E053
:10069E00B4AB61C2AF75D90475B62275F522758FEC
:1006AE000375B7A575B7F1740090F600F0758F015C
:1006BE00755A00755900AE59AF5A7445BE00279F42
:1006CE00402475B7A575B7F19008BC120048E0FC40
:1006DE0090F600120048ECF0785A740126F6500499
:1006EE0018E436F650D0758F0075F51175B6207575
:1006FE00D944D2AF22C2AF75F52275D904755A000E
:10070E00755900AE59AF5A7445BE00229F401F90D6
:10071E00F600120048E493FC9008BC120048ECF07E
:10072E00785A740126F6500418E436F650D575D969
:10073E004475F511D2AF22900071E0B4AA02800385
:10074E00020882C2AF75D90475B62275F522758F6F
:10075E000375B7A575B7F1740090F400F075B7A5E1
:10076E0075B7F1740090F200F075B7A575B7F17416
:10077E000090F000F075B7A575B7F1740090EE001B
:10078E00F0758F01755A00755900AE59AF5A74FF46
:10079E00C39F74019E402475B7A575B7F19000A64E
:1007AE00120048E0FC90F400120048ECF0785A7405
:1007BE000126F6500418E436F650CF755A007559D6
:1007CE0000AE59AF5A74FFC39F74019E402475B793
:1007DE00A575B7F19002A6120048E0FC90F2001247
:1007EE000048ECF0785A740126F6500418E436F6F8
:1007FE0050CF755A00755900AE59AF5A74FFC39F4A
:10080E0074019E402475B7A575B7F19004A6120029
:10081E0048E0FC90F000120048ECF0785A74012683
:10082E00F6500418E436F650CF755A00755900AEDE
:10083E0059AF5A74FFC39F74019E402475B7A575B6
:10084E00B7F19006A6120048E0FC90EE00120048A8
:10085E00ECF0785A740126F6500418E436F650CFB0
:10086E00758F0075F51175B62075D944D2AF743AEF
:10087E009007A6F022900071E0B4AA02800302094C
:10088E00C0C2AF75D90475B62275F522758F037582
:10089E00B7A575B7F1740090EC00F075B7A575B7F4
:1008AE00F1740090EA00F075B7A575B7F174009079
:1008BE00E800F075B7A575B7F1740090E600F07515
:1008CE008F01755A00755900AE59AF5A74FFC39F08
:1008DE0074019E402475B7A575B7F19000A612005D
:1008EE0048E0FC90EC00120048ECF0785A740126B7
:1008FE00F6500418E436F650CF755A00755900AE0E
:10090E0059AF5A74FFC39F74019E402475B7A575E5
:10091E00B7F19002A6120048E0FC90EA00120048DF
:10092E00ECF0785A740126F6500418E436F650CFDF
:10093E00755A00755900AE59AF5A74FFC39F7401B2
:10094E009E402475B7A575B7F19004A6120048E035
:10095E00FC90E800120048ECF0785A740126F6502C
:10096E000418E436F650CF755A00755900AE59AFDB
:10097E005A74FFC39F74019E402475B7A575B7F1D5
:10098E009006A6120048E0FC90E600120048ECF03B
:10099E00785A740126F6500418E436F650CF758F47
:1009AE000075F51175B62075D944D2AF743A90071B
:1009BE00A6F022C2AF75D90475F522755A00755985
:1009CE0000AE59AF5A74FFC39F74019E401F90F43E
:1009DE0000120048E493FC9000A6120048ECF07858
:1009EE005A740126F6500418E436F650D4755A009F
:1009FE00755900AE59AF5A74FFC39F74019E401FC4
:100A0E0090F200120048E493FC9002A6120048EC0B
:100A1E00F0785A740126F6500418E436F650D47560
:100A2E005A00755900AE59AF5A74FFC39F74019E98
:100A3E00401F90F000120048E493FC9004A61200B0
:100A4E0048ECF0785A740126F6500418E436F65045
:100A5E00D4755A00755900AE59AF5A74FFC39F74BE
:100A6E00019E401F90EE00120048E493FC9006A6F3
:100A7E00120048ECF0785A740126F6500418E43649
:100A8E00F650D475F51175D944D2AF74019000EFBC
:100A9E00F0743A9007A6F09009157401F022C2AFD7
:100AAE0075D90475F522755A00755900AE59AF5AAD
:100ABE0074FFC39F74019E401F90EC00120048E427
:100ACE0093FC9000A6120048ECF0785A740126F6BA
:100ADE00500418E436F650D4755A00755900AE59C4
:100AEE00AF5A74FFC39F74019E401F90EA0012001C
:100AFE0048E493FC9002A6120048ECF0785A740178
:100B0E0026F6500418E436F650D4755A007559007E
:100B1E00AE59AF5A74FFC39F74019E401F90E800F8
:100B2E00120048E493FC9004A6120048ECF0785AA8
:100B3E00740126F6500418E436F650D4755A007532
:100B4E005900AE59AF5A74FFC39F74019E401F9057
:100B5E00E600120048E493FC9006A6120048ECF062
:100B6E00785A740126F6500418E436F650D475F50A
:100B7E001175D944D2AF74029000EFF0743A900719
:100B8E00A6F07402900915F02274019000EFF09017
:100B9E0008BDE0903C1EF828287380188016A2A38A
:100BAE00400674029000EFF0800AA2A44006740280
:040BBE009000EFF0C4
:0C3C1E00020BA8020BAA020BAC020BB8B0
:100BC2009000EFE0B40105A231B34002801AD231A5
:100BD2001246CB1209C174019000EFF012039D126C
:100BE2003DBA741B900075F09000EFE0B40206A2CB
:100BF20031B3B34002801AC2311246CB120AAC742E
:100C0200029000EFF012039D123DBA741B90007522
:100C1200F022E54E64046006E59964FF60028031CB
:100C2200A2274004D2278027E54E600874E6254EAD
:100C3200900075F0E54D600874F0254D900075F058
:100C4200E54EB4010280FE754E00754D00C227804C
:100C520002C227E54E903C2AF8282873754E00E51B
:100C620099B4FF03754D01E599B4FE03754D02E594
:100C720099B4FD03754D03E599B4FC03754D04E584
:100C820099B4FA03754D05E599B4FB06754E011248
:100C920046CBE599B4F906754E041246CBE599B4F4
:100CA200F7331246CBC29C74AB900071F012069AD5
:100CB20074AA900071F0900915E0B401051207457D
:100CC2008003120883900071E4F0D29C754E007587
:100CD2004D007599F7E599D394E54007E599C394DA
:100CE200F04002801685994F754E027E017F00E525
:100CF2004FC394E61271728E328F339008B4E4F0CF
:100D0200A3F0E599D394C24007E599C394E6400263
:100D1200802885994F754E0374E5C3954FF5337559
:100D22003200AE32AF33906B26127141E493F87405
:100D320001939008B4C8F0A3C8F0D2990210A2900F
:100D420008C9E0700AA221B35005A222B340028072
:100D52005C9008B4E0FEA3E0FF74FFBE00039F5066
:100D620009EFC39446EE9406402B9008B4E0FEA32C
:100D7200E0FFEFD3946DEE94064009EFC394EEEEDC
:100D8200940640119008B4E0FEA3E0FFEFD394FF75
:100D9200EE940640139008B4E0FEA3E0FF9000A694
:100DA200120048E599F0800385997480119008B487
:100DB200E0FEA3E0FF9000A6120048E599F090083B
:100DC200B41271809008B4E0FEA3E0FFEFB4010614
:100DD200EEB407028003020E9B9007A6E0B43C0229
:100DE2008003020E9BA221B35005A222B3400280CF
:100DF20055C29C12039D9000B3E0900914F0123E7C
:100E0200F5900192E09008CAF0900193E09008CB2F
:100E1200F0900194E09008CCF074AB900071F01265
:100E2200069A74AA900071F0900915E0B4010512B7
:100E320007458003120883900915E09000EFF090B7
:100E42000071E4F08048C29C12019C74009008CAB0
:100E5200F074009008CBF074009008CCF09000B3CE
:100E6200E0900914F0123EF574AB900071F0120696
:100E72009A74AA900071F0120745120883D29C75E9
:100E820099FB7464F5097508001205E480FED29C92
:100E9200754E00754D007599FB0210A29008B4E0E2
:100EA200FEA3E0FFEF4E7006859931753000900881
:100EB200B4E0FEA3E0FF74016F4E701BAC30AD31A5
:100EC200AA32AB33ED2BFBEC3AFA8A068B07900081
:100ED200A6120048E599F09008B41271809008B407
:100EE200E0FEA3E0FF74026F4E7021AC30AD3174AE
:100EF200566D4C7006E54F64E6600280031246CBE5
:100F0200123EF5854F99754E00754D000210A29064
:100F120008B4E0FEA3E0FF9000A6120048E599F0B5
:100F22009008B41271809008B4E0FEA3E0FFAC32E6
:100F3200AD338F028E038C068D07906B6C1271415C
:100F4200E493F9740193FEEAD39EEB994009854F2D
:100F520099754E00754D000210A29008B4E0FEA3F0
:100F6200E0FF9000A6120048E599F09008B41271D3
:100F7200809008B4E0FEA3E0FFEFB40006EEB401F7
:100F82000280030210A2900087E0D394C7400B9026
:100F92000087E0C394C8F550801A900087E0D3948C
:100FA20063400B900087E0C39464F5508006900084
:100FB20087E0F550E55075F002A4FFAEF08F73EFB5
:100FC2009000A61271A3EFFCE0FDEC9000A9127153
:100FD200A3EDFCE0FDEC2DB5500280030210930F4F
:100FE200EF9000A61271A3E573FFE0FCEF9000AA58
:100FF2001271A3ECFFE0FCEFC39CB5500280030228
:101002001093E5739000A81271A3E573FFE0FCEF63
:101012009000AB1271A3ECFFE0FCEF2CB55072E52F
:10102200739000AC1271A3E0C39550900902F0E5F1
:10103200739000AD1271A3E0C39550900903F0E5DF
:10104200739000B01271A3E0C39550900904F0E5CB
:10105200739000B11271A3E0C39550900905F0E5B9
:10106200739000B21271A3E0C39550900906F0E5A7
:10107200739000B31271A3E0C39550900907F01268
:1010820006107599F97464F5097508001205E48073
:10109200FE7599FF7464F5097508001205E480FE77
:0F3C2A00020C5E020D41020E9E020F11020F5C92
:1010A20022E54D903C39F82828730211879008B444
:1010B200E0FEA3E0FF900077120048E0F599900867
:1010C200B41271809008B4E0FEA3E0FF741C6F4E6E
:1010D2007003754D00021187856E99021187900881
:1010E200B4E0FEA3E0FF9000A6120048E0F599EFFD
:1010F200B40107EEB40703754D009008B412718075
:071102000211879008B5E01F
:0F3C39000210AC0210AF0210DA0210E002110507
:10110900903CABF82828738552998067855F998050
:1011190062856199805D8565998058856799805355
:10112900856899804E8569998049856A9980449036
:101139000027E0F599803CA228B340077599FAC2C7
:10114900288017A220B3400575990F800B90007570
:10115900E0F599900075E4F0C2208017856B9980BD
:1011690012856699800D856C9980087599FC8003B4
:03117900754D00B1
:103CAB0002111002111502111A02111F0211240226
:103CBB00112902112E021133021138021140021187
:0D3CCB006502116A02116F02117402117975
:0B117C009008B41271808003123E1531
:033C4800021184E2
:1011870022E537255AFFAE5950010E9000A61200EE
:1011970048E0F538E537255AFFAE5950010E0FBF25
:1011A70000010E9000A6120048E0F539853F3BE5A7
:1011B70038B539058538378041E539D39538401D2D
:1011C700E539C39538853AF0A4FFAEF0E53B8E04C8
:1011D7008F05FF127162ED2538F537801DE538C39D
:1011E7009539853AF0A4FFAEF0E53B8E048F05FFF5
:1011F700127162EDF4042538F53722E539D39538B5
:10120700401DE539C39538853AF0A4FFAEF0E53BBC
:101217008E048F05FF127162ED2538F537801DE5C5
:1012270038C39539853AF0A4FFAEF0E53B8E048FBD
:1012370005FF127162EDF4042538F537229000ACF2
:10124700E0B4017FE56775F00A84FF7E008F37E51C
:101257006775F00A84ADF07C008D3A753F0A7559C1
:1012670005755A24E537C394115005121188800675
:101277009005DBE0F537E537C394F05008E5379084
:101287000099F0800674EF900099F0E56775F00A11
:1012970084FF7E008F37E56775F00A84ADF07C0028
:1012A7008D3A753F0A755905755A5AE537C3941132
:1012B70050051211888006900611E0F537E5379042
:1012C7000070F0229000ACE0B401028003021359D1
:1012D700E56775F00A84FF7E008F37E56775F00ACA
:1012E70084ADF07C008D3A753F0A755905755A36FD
:1012F700E537C39411500512118880069005EDE07B
:10130700F537E537C394F0500585374B8003754BA8
:10131700EFE56775F00A84FF7E008F37E56775F0A4
:101327000A84ADF07C008D3A753F0A755905755AE8
:1013370048E537C39411500512118880069005FFC0
:10134700E0F537E537C394F0500585374C800375D2
:101357004CEF22E55F75F00484FF7E008F37E55F71
:1013670075F00484ADF07C008D3A753F0475590122
:10137700755A00E537C3943F5005121188800690CF
:1013870001E5E0F537E5379008AEF8E4F0E8A3F0BB
:10139700900074E075F020A4FFAEF09000F7E08EA7
:1013A700048F05FF1271628D379000DFE0D3955FE0
:1013B7005003021465900103E0D3955F4010ED9050
:1013C70001E61271A3E0F52B752A00021462900062
:1013D700CEE0D3955F4043E5379001E61271A3E075
:1013E700F538E5379002061271A3E0F5399001034D
:1013F700E0F404255FF53A9000CEE0FE900103E0AB
:10140700F4042EF53BE538B53905853837800312E6
:10141700120285372B752A008041E53790020612A4
:1014270071A3E0F538E5379002261271A3E0F5398C
:101437009000CEE0F404255FF53A9000DFE0FE90DF
:1014470000CEE0F4042EF53BE538B539058538378D
:10145700800312120285372B752A0002150C9001A2
:1014670006E0D3955F5011E5379002661271A3E04D
:10147700F52B752A0002150C9000CFE0D3955F502D
:1014870043E5379002461271A3E0F538E53790023D
:10149700661271A3E0F5399000CFE0F404255FF5FB
:1014A7003A900106E0FE9000CFE0F4042EF53BE50C
:1014B70038B53905853837800312120285372B7501
:1014C7002A008041E5379002261271A3E0F538E53E
:1014D700379002461271A3E0F5399000DFE0F4047B
:1014E700255FF53A9000CFE0FE9000DFE0F4042E90
:1014F700F53BE538B5390585383780031212028583
:10150700372B752A0022900117E0F53C753F1175BE
:101517005902755A00AE51AF52E53C75F00FA4FD64
:10152700ACF0EDD39FEC9E4021E53C8E048F05FF88
:10153700127162ED75F010A4FFAEF0E55F75F01162
:1015470084FD7C00ED2FF53D800EE55F75F011847D
:10155700FF7E00EF24F0F53D853D37E55F75F0111F
:1015670084AFF07E008F3A12118885373EAE51AFB7
:1015770052900117E075F00FA4FDACF0EDD39FEC8E
:101587009E4028755902755A10853D371211888576
:101597003E38853739AE51AF52E53C8E048F05FF93
:1015A70012718D8D3A853C3B121202E5379008AED9
:1015B700F8E4F0E8A3F0752B64752A002290011770
:1015C700E0F53C753F11755902755A00AE51AF529F
:1015D700E53C75F00FA4FDACF0EDD39FEC9E4021E8
:1015E700E53C8E048F05FF127162ED75F010A4FFC4
:1015F700AEF0E56175F01184FD7C00ED2FF53D80BF
:101607000EE56175F01184FF7E00EF24F0F53D854E
:101617003D37E56175F01184AFF07E008F3A121106
:101627008885373EAE51AF52900117E075F00FA491
:10163700FDACF0EDD39FEC9E4028755902755A100A
:10164700853D37121188853E38853739AE51AF52FF
:10165700E53C8E048F05FF12718D8D3A853C3B1258
:101667001202E5379008AEF8E4F0E8A3F0E56B6006
:1016770017E56BC394FE501090010BE0B40209907C
:1016870000F9E0D3940B5002801F9008AEE0FEA350
:10169700E0FFE56B12717274E78E048F05FF12711C
:1016A700629008AEECF0A3EDF09000E1E0B4045FC7
:1016B700E55F75F00484FF7E008F37E55F75F00402
:1016C70084ADF07C008D3A753F04755901755A0059
:1016D700E537C3943F500512118880069001E5E075
:1016E700F5379008AEE0FEA3E0FFE537127172749C
:1016F700328E048F05FF1271629008AEE0FEA3E000
:10170700FFEF2DFDEE3CFC9008AEECF0A3EDF0757D
:101717002B64752A00229000ACE0B40146E567759A
:10172700F00A84FF7E008F37E56775F00A84ADF015
:101737007C008D3A753F0A755905755A00E537C320
:101747009411500512118880069005B7E0F537AE61
:101757002AAF2BE5372FFF50010E74641271B58E37
:101767002A8F2B9000ADE0B40146E56875F00A8436
:10177700FF7E008F37E56875F00A84ADF07C008D39
:101787003A753F0A755905755A6CE537C394115078
:10179700051211888006900623E0F537AE2AAF2B95
:1017A700E5372FFF50010E74641271B58E2A8F2B07
:1017B7009000BCE0B40249E56AC3944175F0058422
:1017C700FF7E008F37E56A75F00584ADF07C008DEC
:1017D7003A753F05755906755A00E537C394135096
:1017E7000512118880069006B9E0F537AE2AAF2BAF
:1017F700E5372FFF50010E74641271B58E2A8F2BB7
:101807009000FEE0B4020280030218BCE55F75F0A9
:101817001584FF7E008F37E55F75F01584ADF07C8A
:10182700008D3A753F15755903755AF4E537C3941A
:101837000B500512118880069004A5E0F537E537AF
:1018470075F0FFA4FFAEF09000FFE08E048F05FF58
:10185700127162ED900095F0E56675F078A4FFAE21
:10186700F074FF8E048F05FF1271628C598D5A74C4
:10187700028C068D071200398F37AC59AD5A7404A4
:10188700FF12718D8D3A753F04755906755A28E513
:1018970037C3941D500512118880069006EBE0F5BA
:1018A70037AE2AAF2BE5372FFF50010E7464127144
:1018B700B58E2A8F2B9000ABE0B4025DE56175F021
:1018C70064A4FFAEF074081200398E5B8F5C740558
:1018D7008E048F05FF1271628D37AE5BAF5C7405A6
:1018E7008E048F05FF12718D8D3A753F0575590569
:1018F700755ADEE537C39413500512118880069098
:101907000697E0F537AE2AAF2BE5372FFF50010ECC
:1019170074641271B58E2A8F2B9000EDE0707F9062
:101927000074E075F00A84FF7E008F37900074E042
:1019370075F00A84ADF07C008D3A753F0A7559053C
:10194700755AC0E537C3940E50051211888006906A
:101957000674E0F537E53790009AF090010CE0B493
:10196700023C900074E075F00A84FF7E008F379088
:101977000074E075F00A84ADF07C008D3A753F0A7B
:10198700755905755ACFE537C3940E50051211885E
:101997008006900683E0F537E53790009BF02290AC
:1019A70000B4E0B40117900909E0252BFFAE2A50D7
:1019B700010E900108E01271B58E2A8F2B90012C31
:1019C700E0B4011490012DE0A851B80004955250DD
:1019D70007E55FC39560400280139000D6E0252B92
:1019E700FFAE2A50010E8E2A8F2B021E0D9000B4D7
:1019F700E0B40306A225B3B340028050900913E078
:101A0700701090090CE0C39405A851B800069552D0
:101A1700400280109000D6E0252BFFAE2A50010E21
:101A27008E2A8F2B900913E0600D90090CE0A851C6
:101A3700B800069552400280109000D6E0252BFF93
:101A4700AE2A50010E8E2A8F2B021E0D9000AEE09B
:101A5700B402028003021E0D9000B1E0602FE5671B
:101A6700D39446402890001EE0FEA3E0FF9000ECD0
:101A7700E075F003A4FDACF0EFD39DEE9C400E9013
:101A87000110E0A851B80005D395525003021E0D6E
:101A97009000E1E0B403028003021C5585615A758A
:101AA70059009000B8E0A851B800049552500E9024
:101AB70000B9E0A859B80005D3955A5003021C5243
:101AC700E56175F002A4FFAEF074158E048F05FF73
:101AD7001271628C068D07900636120048FEE0FFF1
:101AE700EE9000B0E0FEEF8E0088F0A4FFAEF07439
:101AF700648E048F05FF1271628C598D5A900074A1
:101B0700E075F018A4FFAEF09000F7E08E048F05A3
:101B1700FF1271628C068D0790064E120048AE596F
:101B2700AF5AE012717274648E048F05FF127162EE
:101B37008C598D5AE565A859B80005D3955A5003B5
:101B4700021BC9E565C3955AFFE49559FE8E598F67
:101B57005A7428BE00039F500C755A287559007493
:101B67000D900075F0AE59AF5A9000B1E012717246
:101B770074288E048F05FF1271628C598D5A900854
:101B8700AEE0FEA3E0FF740A8E048F05FF127162B8
:101B97008D068C07AC59AD5ACFCECF120003740A0D
:101BA7008E048F05FF1271628C598D5A9008AEE032
:101BB700FEA3E0FF1271BD9008AEEEF0A3EFF002B6
:101BC7001C52E565A859B80004955A507EAE59AF26
:101BD7005AE5651271B58E598F5A7428BE00039F56
:101BE700500C755A28755900740D900075F0AE5950
:101BF700AF5A9000B1E012717274288E048F05FFFE
:101C07001271628C598D5A9008AEE0FEA3E0FF7402
:101C17000A8E048F05FF1271628D068C07AC59ADD1
:101C27005ACFCECF120003740A8E048F05FF1271AC
:101C3700628C598D5A9008AEE0FEA3E0FFEF2DFDB0
:101C4700EE3CFC9008AEECF0A3EDF0021E0D900008
:101C5700F9E0855FF0A4FFAEF074051271727407A6
:101C67001200398E598F5A9000B8E0A851B8000475
:101C7700955250129000B9E075F002A4FDACF0EF58
:101C8700C39DEE9C4003021E0DE55F75F00B84FFBC
:101C97007E00900636120048FEE0FFEE9000B0E0AE
:101CA700FEEF8E0088F0A4FFAEF074648E048F05FB
:101CB700FF1271628C598D5A900074E075F018A468
:101CC700FFAEF09000F7E08E048F05FF1271628C73
:101CD700068D0790064E120048AE59AF5AE01271B2
:101CE7007274648E048F05FF1271628C598D5AE5E8
:101CF70065A859B80005D3955A5003021D84E565B8
:101D0700C3955AFFE49559FE8E598F5A7428BE0021
:101D1700039F500C755A28755900740D900075F083
:101D2700AE59AF5A9000B1E012717274288E048FC9
:101D370005FF1271628C598D5A9008AEE0FEA3E040
:101D4700FF740A8E048F05FF1271628D068C07AC33
:101D570059AD5ACFCECF120003740A8E048F05FFF8
:101D67001271628C598D5A9008AEE0FEA3E0FF1203
:101D770071BD9008AEEEF0A3EFF0021E0DE565A869
:101D870059B80004955A507EAE59AF5AE56512719D
:101D9700B58E598F5A7428BE00039F500C755A2868
:101DA700755900740D900075F0AE59AF5A9000B197
:101DB700E012717274288E048F05FF1271628C59BC
:101DC7008D5A9008AEE0FEA3E0FF740A8E048F05DB
:101DD700FF1271628D068C07AC59AD5ACFCECF1268
:101DE7000003740A8E048F05FF1271628C598D5A95
:101DF7009008AEE0FEA3E0FFEF2DFDEE3CFC90085F
:101E0700AEECF0A3EDF02290010CE0B4027BE55FAD
:101E170075F00884FF7E008F37E55F75F00884ADA5
:101E2700F07C008D3A753F08755901755AE0E53722
:101E3700C3943F500512118880069002A5E0F5373C
:101E4700E5379008B0F8E4F0E8A3F09008B0E0FEBA
:101E5700A3E0FFAC2AAD2B12000374648E048F0538
:101E6700FF1271629008B0ECF0A3EDF09000A9E0CA
:101E77008C068D0712717274648E048F05FF1271C0
:101E8700629008B0ECF0A3EDF09008AEE0FEA3E09E
:101E9700FFAC2AAD2B12000374648E048F05FF126A
:101EA70071629008AEECF0A3EDF09000A9E08C060B
:101EB7008D0712717274648E048F05FF1271629020
:101EC70008AEECF0A3EDF0A203401DAE51AF527483
:101ED70005BE00039F5002D203E561D394CC4008AE
:101EE700D2017411900075F02290010BE0B4020842
:101EF7009000F9E0640B600280459008AEE0FEA315
:101F0700E0FFE56B12717274E78E048F05FF1271A3
:101F1700629008AEECF0A3EDF090010CE0B4021F64
:101F27009008B0E0FEA3E0FFE56B12717274E78ED4
:101F3700048F05FF1271629008B0ECF0A3EDF090EA
:101F470000CBE05402601B9000C2E0A851B8001219
:101F5700D39552400DA203B3B35007E561C3949ADA
:101F67004002805FAE34AF359000C0E075F002A448
:101F7700FDACF0EF2DFDEE3CFC74022DFD50010C85
:101F8700E561BC003ED39D403A754301A22C403326
:101F97009000C1E075F05EA4FDACF07405FF12710E
:101FA700628C5B8D5C1249749008AEE0FEA3E0FF83
:101FB7009000C1E02FFF50010E9008AEEEF0A3EFA6
:101FC700F0D22CE561A834B8000495355002C22C34
:101FD700856135753400E54370030220E690011EE4
:101FE700E0C3954350030220D890012EE0C394022A
:101FF7004003022082E56775F00A84FF7E009005A2
:10200700A6120048E0F55A755900AE59AF5A90002C
:10201700C1E012717274648E048F05FF1271628CB5
:102027005B8D5C90011EE004C395438C068D0712FF
:10203700717290011EE08E048F05FF1271628C5B36
:102047008D5C9008AEE0FEA3E0FFEF2DFDEE3CFCBB
:102057009008AEECF0A3EDF090010CE0B4021A90FA
:1020670008B0E0FEA3E0FFAA5BAB5CEF2BFBEE3A08
:10207700FA9008B0EAF0A3EBF0805690011EE00456
:10208700C39543854BF0A4FFAEF090011EE08E048C
:102097008F05FF1271628C5B8D5C9008AEE0FEA32A
:1020A700E0FFEF2DFDEE3CFC9008AEECF0A3EDF069
:1020B70090010CE0B4021A9008B0E0FEA3E0FFAA7A
:1020C7005BAB5CEF2BFBEE3AFA9008B0EAF0A3EBC0
:1020D700F0054390011EE0C39543500375430090FC
:1020E70000CBE05401601B9000BFE0A851B800127C
:1020F700D39552400DA203B3B35007E55FC394CC09
:10210700400280609000BDE075F003A4FFAEF0E5EB
:10211700402FFF50010E74032FFF50010EE55FBEE5
:102127000042D39F403E754401A22C40379000BE29
:10213700E075F05EA4FFAEF074058E048F05FF1204
:1021470071628C5B8D5C1249749008AEE0FEA3E06F
:10215700FF9000BEE02FFF50010E9008AEEEF0A3F7
:10216700EFF0D22CE55FC395405002C22C855F404B
:10217700E544700302228090011FE0C39544500399
:1021870002227290012EE0C39402400302221CE552
:102197006775F00A84FF7E009005A6120048E0F5F7
:1021A7005A755900AE59AF5A9000BEE01271727459
:1021B700648E048F05FF1271628C5B8D5C90011F2A
:1021C700E004C395448C068D0712717290011FE0DD
:1021D7008E048F05FF1271628C5B8D5C9008AEE0F8
:1021E700FEA3E0FFEF2DFDEE3CFC9008AEECF0A364
:1021F700EDF090010CE0B4021A9008B0E0FEA3E005
:10220700FFAA5BAB5CEF2BFBEE3AFA9008B0EAF063
:10221700A3EBF0805690011FE004C39544854CF072
:10222700A4FFAEF090011FE08E048F05FF127162CC
:102237008C5B8D5C9008AEE0FEA3E0FFEF2DFDEE1A
:102247003CFC9008AEECF0A3EDF090010CE0B4027A
:102257001A9008B0E0FEA3E0FFAA5BAB5CEF2BFB94
:10226700EE3AFA9008B0EAF0A3EBF0054490011FAC
:10227700E0C3954450037544009008AEE0FEA3E028
:10228700FF9000D0E0BE00039F500D9000D0E0907B
:1022970008AEF8E4F0E8A3F090010CE0B402129065
:1022A70008B0E0FEA3E0FF9000D0E0BE00059F402D
:1022B70002800D9000D0E09008B0F8E4F0E8A3F0B9
:1022C7002290010CE0B401028003022416A203B39A
:1022D70050030223FD9000D7E0B4017A9008AEE0E6
:1022E700FEA3E0FFAC51AD52120003743C8E048F85
:1022F70005FF1271629000E7E0BC00159D40129047
:1023070008AEE0FEA3E0FF9000E9E0BE00039F50A7
:1023170002D2029008AEE0FEA3E0FFAC51AD52122C
:102327000003743C8E048F05FF1271629000E7E092
:10233700C3940ABC001AD39D40169008AEE0FEA3D2
:10234700E0FF9000E9E0C39405BE0004D39F50026C
:102357008002C202807A9008AEE0FEA3E0FFAC5193
:10236700AD5212000374788E048F05FF12716290CC
:1023770000E7E0BC00159D40129008AEE0FEA3E028
:10238700FF9000E9E0BE00039F5004D20280419015
:1023970008AEE0FEA3E0FFAC51AD52120003747823
:1023A7008E048F05FF1271629000E7E0C3940ABCA8
:1023B700001AD39D40169008AEE0FEA3E0FF900000
:1023C700E9E0C39405BE0004D39F50028002C20215
:1023D700A202B340219008AEE0FEA3E0FF9000E820
:1023E700E012717274648E048F05FF127162900897
:1023F700AEECF0A3EDF0A202B3400CA2304006749D
:1024070024900075F0D230A2024002C2308002C28E
:1024170002900070E06006A203B3B34002801990F7
:1024270008AEE0FEA3E0FF900070E02FFF50010E22
:102437009008AEEEF0A3EFF0A200B34006A201B3FE
:10244700B35009900026E4F0A3F0802D9008AEE089
:10245700FEA3E0FF7400D39F74019E40119008AE65
:10246700E0F8A3E0900026C8F0A3C8F0800B74FF43
:10247700900026F8E4F0E8A3F09000EEE0C394049F
:10248700400C900910E0C3940240030225709000AD
:10249700D7E0B401479008AEE0FEA3E0FF745E12F8
:1024A700717274058E048F05FF1271629008AEEC8D
:1024B700F0A3EDF090010CE0B4021F9008B0E0FE2D
:1024C700A3E0FF745E12717274058E048F05FF120C
:1024D70071629008B0ECF0A3EDF080459008AEE093
:1024E700FEA3E0FF745E127172740A8E048F05FFFB
:1024F7001271629008AEECF0A3EDF090010CE0B41D
:10250700021F9008B0E0FEA3E0FF745E12717274C0
:102517000A8E048F05FF1271629008B0ECF0A3EDEC
:10252700F09008AEE0FEA3E0FF7402BE000CD39F5C
:102537004008752902752800800A9008AEE0F52842
:10254700A3E0F5299008B0E0FEA3E0FF7402BE0007
:102557000CD39F4008752D02752C00800A9008B097
:10256700E0F52CA3E0F52D80469008AEE0FEA3E051
:10257700FF7401BE000CD39F400875290175280020
:10258700800A9008AEE0F528A3E0F5299008B0E0AE
:10259700FEA3E0FF7401BE000CD39F4008752D0118
:1025A700752C00800A9008B0E0F52CA3E0F52D907B
:1025B7000024E528F0A3E529F0A233B34009C200BF
:1025C700900026E4F0A3F022900074E09003A61296
:1025D70071A3E0F541754264900074E0FE9000E25B
:1025E700E0D39E4037E55F75F00884FF7E008F37A4
:1025F700E55F75F00884ADF07C008D3A753F08758E
:102607005903755A96E537C3941F500512118880F0
:102617000690045BE0F5378537428035E55F75F056
:102627000884FF7E008F37E55F75F00884ADF07C86
:10263700008D3A753F08755903755AB6E537C39447
:102647001F5005121188800690047BE0F537853707
:102657004222900118E0F53C753F11755904755AEF
:1026670000AE51AF52E53C75F00FA4FDACF0EDD3D1
:102677009FEC9E4021E53C8E048F05FF127162EDB1
:1026870075F010A4FFAEF0E55F75F01184FD7C00D6
:10269700ED2FF53D800EE55F75F01184FF7E00EFAD
:1026A70024F0F53D853D37E55F75F01184AFF07E89
:1026B700008F3A12118885373EAE51AF52900118FC
:1026C700E075F00FA4FDACF0EDD39FEC9E402875AC
:1026D7005904755A10853D37121188853E3885375C
:1026E70039AE51AF52E53C8E048F05FF12718D8DC7
:1026F7003A853C3B121202853741754264229001AC
:1027070018E0F53C753F11755904755A00AE51AF85
:1027170052E53C75F00FA4FDACF0EDD39FEC9E4065
:1027270021E53C8E048F05FF127162ED75F010A450
:10273700FFAEF0E56175F01184FD7C00ED2FF53DEE
:10274700800EE56175F01184FF7E00EF24F0F53D02
:10275700853D37E56175F01184AFF07E008F3A1241
:10276700118885373EAE51AF52900118E075F00FD2
:10277700A4FDACF0EDD39FEC9E4028755904755A23
:1027870010853D37121188853E38853739AE51AFF0
:1027970052E53C8E048F05FF12718D8D3A853C3BC7
:1027A700121202853741754264900113E0B404792F
:1027B700900074E0FE9000E2E0D39E4037E55F753D
:1027C700F00884FF7E008F37E55F75F00884ADF071
:1027D7007C008D3A753F08755903755A96E537C3DE
:1027E700941F5005121188800690045BE0F5378529
:1027F70037428035E55F75F00884FF7E008F37E547
:102807005F75F00884ADF07C008D3A753F08755907
:1028170003755AB6E537C3941F5005121188800611
:1028270090047BE0F537853742229000ACE0B40195
:102837003BE56775F00A84FF7E008F37E56775F023
:102847000A84ADF07C008D3A753F0A755905755AB3
:1028570012E537C39411500512118880069005C9F7
:10286700E0F537E5422537C39464F5429000ADE0C3
:10287700B4013BE56875F00A84FF7E008F37E56891
:1028870075F00A84ADF07C008D3A753F0A755905DD
:10289700755A7EE537C3941150051211888006904A
:1028A7000635E0F537E5422537C39464F542E5413F
:1028B7002542F5369000B4E0B40210900908E025EF
:1028C70036FE900108E0F4042EF53690010BE0D3B4
:1028D70094014040E56BC394E7501D74E7C3956BC3
:1028E700FE90090AE08E00F5F0E884FF7E008F373E
:1028F700E5362537F536801CE56BC394E7FE90096E
:102907000AE08E00F5F0E884FF7E008F37E536C3D6
:102917009537F536A2034006E5412464F536E536DA
:10292700D394644009E536C39464F536800375365D
:10293700009000E4E0C3953650069000E4E0F536D9
:1029470022D200900098E0A851B800049552503E5A
:10295700900098E0A851B800049552500375360FBF
:10296700900098E004A851B80004955250037536BA
:1029770007900098E02402A851B80004955250022D
:10298700C200900098E060067409900075F0C22BB1
:102997007E017F009000EAE01271729000F9E08EEC
:1029A700048F05FF127162E55FBC000CD39D4008E0
:1029B700D233740A900075F09000ACE0B40109902E
:1029C70000EBE0C39567400280159000FDE0A85139
:1029D700B8000495525002C200740B900075F09035
:1029E70000ACE0B40107E567C394644002801D9022
:1029F7000143E0600D900143E0A851B800069552ED
:102A070040028008C200740B900075F0A2004003DA
:102A1700753600C23290012CE0B4011490012DE00C
:102A2700A851B8000495525007E55FC3956040026E
:102A3700802A9000D5E0D3941D400B9000D5E0C3C9
:102A4700941EF5368003753600A22F400874159042
:102A57000075F0D232D22FD22D022B42C22DC22FB7
:102A67009000B4E0B40306A225B3B34003022B429F
:102A770090090CE0C39405A851B80004955250067C
:102A8700900913E06002801F9000D5E0D3941D40A9
:102A97000B9000D5E0C3941EF5368003753600749D
:102AA7000C900075F0D23290090CE0A851B80004E0
:102AB70095525006900913E07002801F9000D5E0F0
:102AC700D3941D400B9000D5E0C3941EF5368003C8
:102AD700753600740C900075F0D23290090CE0A89E
:102AE70051B80004955250319000F3E0B40228D257
:102AF7002B900912E0FE900913E0D39E500690092F
:102B070013E070028009900912E4F0C22B8006904E
:102B17000912E004F08002C20090090CE02405A825
:102B270051B80004955250139000F3E0B4020A9094
:102B37000913E07002D22B8002C200A22AB34027F9
:102B47009000D5E0D3941D400B9000D5E0C3941EB0
:102B5700F5368003753600A22E4006741090007576
:102B6700F0D22ED2328002C22E85366C9000D5E08C
:102B7700D3941D40189000A3E02536FE900074E022
:102B870075F01E84FC7F00EE2CF5368029A232B347
:102B970040089000A3E0F536801C9000A5E025369C
:102BA700FE9000A3E02EFE900074E075F01E84FCFA
:102BB7007F00EE2CF536A233B34005D22B756C009F
:102BC70022900074E075F00584FF7E008F37900037
:102BD70074E075F00584ADF07C008D3A753F05759E
:102BE7005903755AD69000F7E01475F00584FF7EF7
:102BF70000E537BE00039F5005121188800BE537AB
:102C070090047C1271A3E0F537E53790090BF0903B
:102C1700090BE0FE9000E6E0C39E50089000E6E056
:102C270090090BF09000D5E0D3941D401E90090B3E
:102C3700E0FE9000A3E02EFE900074E075F01E8485
:102C4700FC7F00EE2C90090BF08031A232B3400AD2
:102C57009000A3E090090BF0802290090BE0FE9012
:102C670000A5E02EFE9000A3E02EFE900074E07514
:102C7700F01E84FC7F00EE2C90090BF0229000AC34
:102C8700E0B40136E56775F00A84FF7E009005A67B
:102C9700120048E0F546E546D394644010E546C384
:102CA700946475F00F84FF7E008F4680037546009D
:102CB7009000C9E02546F54680069000C9E0F54634
:102CC70022E56775F00A84FF7E009005A61200488A
:102CD700E0C394694007E567D394644055900113B6
:102CE700E0C3940350269008A8E0FEA3E0FF740415
:102CF700120039E55F127172740F8E048F05FF128F
:102D070071629008A6ECF0A3EDF080249008A8E08B
:102D1700FEA3E0FF7404120039E561127172740FAB
:102D27008E048F05FF1271629008A6ECF0A3EDF0F8
:102D3700800F9008A8E0F8A3E09008A6C8F0A3C801
:102D4700F0A203401A9008A8E0FEA3E0FF74031264
:102D5700717274011200399008A6EEF0A3EFF0909B
:102D670000BCE0B40262E56AC3944175F00584FFD4
:102D77007E008F37E56A75F00584ADF07C008D3AEB
:102D8700753F05755906755A14E537C394175005ED
:102D970012118880069006CDE0F5379008A6E0FE70
:102DA700A3E0FF740A8E048F05FF127162E5378C6A
:102DB700068D07127172740A8E048F05FF127162F5
:102DC7009008A6ECF0A3EDF09008A6E0FEA3E0FFC4
:102DD7009008ACE0FCA3E0FDEDD39FEC9E400F9084
:102DE70008ACE0F8A3E09008A6C8F0A3C8F022E575
:102DF7000875F004A4FFAEF09006E9120048E090D1
:102E07003C4BF8282873804C85527380479000F913
:102E1700E0855FF0A4FFAEF074081200398F73806D
:102E270033856173802E8567738029856873802455
:102E3700856973801F856A73801A856B7380158512
:102E470066738010856573800B856C7380069000B0
:042E570027E0F57308
:103C4B00022E0D022E0F022E14022E28022E2D02F2
:103C5B002E32022E37022E3C022E41022E46022E0F
:073C6B004B022E50022E5502
:102E5B00E50875F004A4FFAEF09006EA120048E511
:102E6B000875F004A4FFAEF0E0FC9006EB120048EE
:102E7B00ECFEE0FFEEC39F4003022F63E50875F005
:102E8B0004A4FFAEF09006E9120048E0B40441E55B
:102E9B000875F004A4FFAEF09006EB120048E0C3F7
:102EAB009573500AE508F50CD39234123D5CE50896
:102EBB0075F004A4FFAEF09006EA120048E0D3953B
:102ECB0073400AE508F50CC39234123D5C022F6186
:102EDB00E50875F004A4FFAEF09006EA120048E096
:102EEB00C395735015E50875F004A4FFAEF090067A
:102EFB00EB120048E0D395735002800AE508F50CFD
:102F0B00D39234123D5CE50875F004A4FFAEF0904B
:102F1B0006EA120048E0D395735015E50875F004E6
:102F2B00A4FFAEF09006EB120048E0C39573500A75
:102F3B00E508F50CC39234123D5C9006F1E0B40148
:102F4B0009900105E0D395615002800A7402F50CDB
:102F5B00C39234123D5C806AE50875F004A4FFAEA1
:102F6B00F09006EA120048E0D395734015E508751A
:102F7B00F004A4FFAEF09006EB120048E0C395738B
:102F8B004002800AE508F50CC39234123D5CE5085B
:102F9B0075F004A4FFAEF09006EA120048E0C3956A
:102FAB00734015E50875F004A4FFAEF09006EB1224
:102FBB000048E0D39573400AE508F50CD392341220
:102FCB003D5C22AE2EAF2F74C9BE000CD39F4008C0
:102FDB00782E1271C50230E8752F01752E00AE5197
:102FEB00AF52E546BE000DD39F40099000DBE0D306
:102FFB00954740028023754700E546C39552F5730C
:10300B009000DEE0D395454008E5452573F54580F6
:10301B00069000DEE0F545800205479000B7E0D34F
:10302B009561401CE55FC395604015AE51AF52E50D
:10303B0046BE00039F50099000DCE0D39548400248
:10304B00806E90090DE0A851B8000495525003759D
:10305B004A0090090DE0A851B8000BD395524006D9
:10306B00E55290090DF0E54A7041E552C39546F5DE
:10307B0073E573D3940540037573059000DDE0C3CE
:10308B0095455007E573C3954540028009E545C357
:10309B009573F54580069000DDE0F5459000DDE089
:1030AB00D3954540069000DDE0F54575480080025C
:1030BB000548E54A70169000B7E0C39561500DE5E1
:1030CB00462405A851B8000695524002800F900087
:1030DB00CAE0F545754A01747890090DF022AE2EC1
:1030EB00AF2F74E9D39F74039E4008782E1271C5DD
:1030FB0002328F752F01752E00754532A226402A9C
:10310B007545199000CAE075F002A4FFAEF0E547D3
:10311B00BE0006D39F4002D2260547754A0374783A
:10312B0090090DF0754900023276AE51AF52E5466B
:10313B006F4E7003023276E546BE000DD39F4009F9
:10314B009000DBE0D395474002800F754700E54ABE
:10315B00C394035003754519800DE546C39552F58D
:10316B0073E5472573F5479000B7E0D39561400EA3
:10317B0090090DE0A851B80007D395524002800C7E
:10318B0005499000CAE0B54903754A00E54AB40306
:10319B0006A203B3B34002800A0549E549B43C03D8
:1031AB00754A02E54AB4022990090DE0A851B8000E
:1031BB000ED395524009E55290090DF075490090D8
:1031CB0000B7E0C395615009754900747890090DFB
:1031DB00F0E54A705A9000B7E0D39561401CE55F6B
:1031EB00C395604015AE51AF52E546BE00039F50EC
:1031FB00099000DCE0D395484002800875480075C3
:10320B00454B8028E552C39546F573E573D394057A
:10321B0040037573059000B7E0D395614008E5480E
:10322B002573F5488006E5482406F548754900E501
:10323B004A70169000B7E0C39561500DE546240522
:10324B00A851B80006955240028003754A01E54A21
:10325B00B4011875451905499000CAE0B5490675C2
:10326B004A02754900747890090DF0A201B340032E
:10327B00754532E54575F00AA4FFAEF09008B2EE45
:10328B00F0A3EFF022E56F903C72F8282873023C14
:10329B000B9000AFE070030235BA9000E5E0B4018B
:1032AB00028003023450900072E0655E6009E552C3
:1032BB004551600302344D7E017F00E5BE127172F1
:1032CB00E5BD2FFF50010E8E598F5A9000E3E0B4ED
:1032DB00461B740E127172900097E08E048F05FFDF
:1032EB001271629008B6ECF0A3EDF0801DAE59AFF1
:1032FB005A7410127172900097E08E048F05FF12B2
:10330B0071629008B6ECF0A3EDF0E56B600FE56B26
:10331B00C394FE500890010BE0640260028064903D
:10332B0000F9E0B40B1F9008B6E0FEA3E0FF74E7D2
:10333B00127172E56B8E048F05FF1271629008B6E5
:10334B00ECF0A3EDF09000F9E0D3940B4008900063
:10335B00E1E064046002802B9008B6E0FEA3E0FF7E
:10336B009008BAE0FCA3E0FDEFD39DEE9C400D125C
:10337B0071BD9008B6EEF0A3EFF080079008B6E4AD
:10338B00F0A3F09008B6E0FEA3E0FFEFD39400EEBD
:10339B0094014008D2337426900075F0A233B3B376
:1033AB00502C7E057F009000F9E08E048F05FF12F4
:1033BB0071629008B6E0FEA3E0FFEFC39DEE9C4068
:1033CB000FAC51AD52740FBC0004D39D5002800260
:1033DB00C2339000AFE0B402279008B8E0FEA3E040
:1033EB00FF9008B6E0FCA3E0FDEF2DFDEE3CFC7476
:1033FB00018C068D071200399008B6EEF0A3EFF0A2
:10340B009008B6E0FEA3E0FF9008B8E0FCA3E0FD57
:10341B00EDD39FEC9E4004D2298002B2299008B6CE
:10342B00E0F8A3E09008B8C8F0A3C8F09000E1E082
:10343B0064016006A229B3B3400280069008B7E08E
:10344B00F55F0235B8D2297E017F00E5BE1271729D
:10345B00E5BD2FFF50010E8E598F5A9000E3E0B45B
:10346B00461B740E127172900097E08E048F05FF4D
:10347B001271629008B6ECF0A3EDF0801DAE59AF5F
:10348B005A7410127172900097E08E048F05FF1220
:10349B0071629008B6ECF0A3EDF0E56B600FE56B95
:1034AB00C394FE500890010BE064026002806490AC
:1034BB0000F9E0B40B1F9008B6E0FEA3E0FF74E741
:1034CB00127172E56B8E048F05FF1271629008B654
:1034DB00ECF0A3EDF09000F9E0D3940B40089000D2
:1034EB00E1E064046002802B9008B6E0FEA3E0FFED
:1034FB009008BAE0FCA3E0FDEFD39DEE9C400D12CB
:10350B0071BD9008B6EEF0A3EFF080079008B6E41B
:10351B00F0A3F09008B6E0FEA3E0FFEFD39400EE2B
:10352B0094014008D2337426900075F0A233B3B3E4
:10353B00502C7E057F009000F9E08E048F05FF1262
:10354B0071629008B6E0FEA3E0FFEFC39DEE9C40D6
:10355B000FAC51AD52740FBC0004D39D50028002CE
:10356B00C2339000AFE0B402279008B8E0FEA3E0AE
:10357B00FF9008B6E0FCA3E0FDEF2DFDEE3CFC74E4
:10358B00018C068D071200399008B6EEF0A3EFF010
:10359B009008B6E0F8A3E09008B8C8F0A3C8F09084
:1035AB0000E1E0640160069008B7E0F55F80037509
:1035BB005F009000ABE07006756F0302329075BB35
:1035CB0018023C0B023C0B9000ABE070030237433C
:1035DB007E017F00E5BE127172E5BD2FFF50010E1B
:1035EB008E598F5A9000F1E0B4010F7E0F7FFFAC24
:1035FB0059AD5A1271BD8E598F5A900116E0B40213
:10360B0045AE59AF5A900030E0FCA3E0FDEDD39FDF
:10361B00EC9E400A900030E559F0A3E55AF0AE5904
:10362B00AF5A900032E0FCA3E0FDEFD39DEE9C403F
:10363B000A900032E559F0A3E55AF0AE59AF5A742F
:10364B00041200398F61900116E0704CAE59AF5ADD
:10365B00900030E0FCA3E0FDEFD39DEE9C400912FF
:10366B0071BD8E598F5A8006755A00755900AE5927
:10367B00AF5A7410127172900115E08E048F05FF12
:10368B001271628C598D5A74FFBC0009D39D400591
:10369B00855A6180037561FE9000E1E0B401028000
:1036AB0003023741A203B3B3500E9000B5E0A8510B
:1036BB00B80005D39552500280719000F2E08561FD
:1036CB00F0A4FFAEF074648E048F05FF1271628C50
:1036DB00598D5AE56B6016E56BC394FE500F900144
:1036EB000BE0B402089000F9E0640B60028017AEA7
:1036FB0059AF5A74E7127172E56B8E048F05FF1286
:10370B0071628C598D5AAE59AF5A9008B6E0FCA332
:10371B00E0FDEDD39FEC9E4005855A5F800BA229FF
:10372B00B340069008B7E0F55F800BA229B34006C3
:10373B009008B7E0F55F80037561009000AEE07014
:10374B0006756F0502329075BB19023C0B023C0BE0
:10375B009000AEE070030237FBE55ED3955D40034E
:10376B000237F990002EE0FEA3E0FFE5651271B57C
:10377B0090002EEEF0A3EFF07E017F00E5BE1271FC
:10378B0072E5BD2FFF50010E8E598F5A90011BE031
:10379B007013740A12717274518E048F05FF1271BB
:1037AB00628D658019AE59AF5A740A1271728F040B
:1037BB008E057E017F95CDCCCD1270608F65E56552
:1037CB00D39464400375656490002EE0FEA3E0FF84
:1037DB00E5652FFF50010E90002EEEF0A3EFF09059
:1037EB0000B2E0048E048F05FF1271628D658003B9
:1037FB007565329000FEE07006756F0702329075AA
:10380B00BB13023C0B023C0B9000FEE0604A7E01B6
:10381B007F00E5BE127172E5BD2FFF50010E8E5970
:10382B008F5A74041200398F66900100E08566F0A0
:10383B00A4FDACF07464FF1271628D669000FFE022
:10384B008566F0A4FFAEF074FF8E048F05FF127136
:10385B0062ED900096F080037566009000ACE0700E
:10386B0006756F0902329075BB17023C0B023C0BBD
:10387B009000ACE0B40102800302390F7E017F009F
:10388B00E5BE127172E5BD2FFF50010E8E598F5A96
:10389B0090090EE0601990090EE014906BB21200C3
:1038AB008CE493FC740193FDEDC39FEC9E4002806E
:1038BB000690090EE014F090090EE0C394B3501D6E
:1038CB00AE59AF5A90090EE004906BB212008CE423
:1038DB0093FC740193FDEFC39DEE9C400280069018
:1038EB00090EE004F090090EE0FE9000D2E08E008D
:1038FB0088F0A4FFAEF074648E048F05FF12716222
:10390B008D6780037567009000ADE07006756F0BD7
:10391B0002329075BB16023C0B023C0B9000ADE0E3
:10392B00B4010280030239BB7E017F00E5BE127138
:10393B0072E5BD2FFF50010E8E598F5A90090FE083
:10394B00601990090FE014906D1C12008CE493FC2D
:10395B00740193FDEDC39FEC9E4002800690090F0E
:10396B00E014F090090FE0C394B3501DAE59AF5A59
:10397B0090090FE004906D1C12008CE493FC740111
:10398B0093FDEFC39DEE9C4002800690090FE0046F
:10399B00F090090FE0FE9000D8E08E0088F0A4FFB5
:1039AB00AEF074648E048F05FF1271628D68800314
:1039BB0075680075BB1F023C0B023C0B7E017F0040
:1039CB00E5BE127172E5BD2FFF50010E8E598F5A55
:1039DB00740912717274E68E048F05FF1271628D79
:1039EB006A9000B4E07006756F0F02329075BB15CC
:1039FB00023C0B023C0B9000B4E07003023B527E86
:103A0B00017F00E5BE127172E5BD2FFF50010E8ED6
:103A1B00598F5A74041200398F699000B4E0B401C5
:103A2B0015900108E08569F0A4FFAEF07407120051
:103A3B0039EF900909F09000B4E0B4021590010839
:103A4B00E08569F0A4FFAEF07407120039EF90091E
:103A5B0008F09000B4E0B403028003023B35900001
:103A6B00F5E07052E569C39419500FD2259000D43C
:103A7B00E090090CF0900911E4F0E569D3946440EF
:103A8B0004A2254002802D900911E004F090091149
:103A9B00E0FE900147E0B5060B90090CE004F090B6
:103AAB000911E4F090090CE064966006900147E080
:103ABB007002C22580639000D4E07034900108E05E
:103ACB008569F0A4FFAEF074FF8E048F05FF1271B1
:103ADB0062ED90090CF0AE51AF52741EBE0006D3CE
:103AEB009F4002D225E561D394E54002C22580298F
:103AFB00E569C3940A500DAE51AF52741EBE00045B
:103B0B00D39F50028002D225E561D394E54002C2D7
:103B1B00259000D4E090090CF090090CE0C39405BB
:103B2B005006740590090CF0C22A9000B4E0B4045E
:103B3B0014E569C394195002D22AE569D394324033
:103B4B0002C22AC225800375690090010BE0700642
:103B5B00756F1102329075BB14023C0B023C0B903B
:103B6B00010BE07003023BF87E017F00E5BE127192
:103B7B0072E5BD2FFF50010E8E598F5A900130E028
:103B8B007025EFD39421EE940E4005756BFF8015D5
:103B9B00AE59AF5A741012717274E38E048F05FF15
:103BAB001271628D6B8027AE59AF5AEFD39449EEE9
:103BBB0094064005756BFF8015AE59AF5A74101201
:103BCB00717274638E048F05FF1271628D6BE56BDE
:103BDB0075F00BA4FFAEF09000F9E08E048F05FF9B
:103BEB001271629008BAECF0A3EDF08003756B00D4
:103BFB009000AFE0600575BB1A800375BB188000A1
:103C720002329902329C0235CF0235D20237580203
:103C8200375B02381002381302387802387B023967
:103C9200240239270239C40239C70239FE023A0125
:093CA200023B67023B6A023C0B85
:103C0B00E56F75F00284AFF07E00EF4E7002D2ECE0
:033C1B00056F2210
:0971A3002582F5825002058322C9
:0F008C0025E050020583258250020583F582226C
:10714100EF2F500205832582F582E5833E2EF583DC
:01715100221B
:1071B500CFC39FFF50011E22C3EF9DFFEE9CFE2211
:0871C5000806B60002180622BC
:0D718000A3E004F07006127199E004F02203
:0E003900048007C3CE13CECF13CFD5E0F6223E
:10706000BC000FBE0008ED8FF084FFADF022E4FEFF
:10707000FF22BE000DEF60FE54F0606F20E70302B8
:107080007116EAC0E0EBC0E078017A0075F001EE1D
:1070900020E710EF25E0FFEE33FE0AC5F023C5F030
:1070A00030E7F0EA5407F9096A7A007B00600108CA
:1070B000C3EC9E40167004ED9F4010ED9FFDEC9ECA
:1070C000FCE5F0CA4ACA03F5F08005E5F003F5F0E7
:1070D000C3EE13FEEF13FFD9D77908CACBCAD8D0B5
:1070E000EAFEEBFFD0E0FBD0E0FA22EC8FF084FC6C
:1070F000ED54F045F0C48FF084FEEDC454F045F03B
:10710000C48FF084FDEEC4FE54F02DFFEE540F3C0E
:10711000FEADF07C0022790078008FF0EC7E082034
:10712000E70DC3CD33CD33C933C9C833C8DEF084CE
:1071300049F9E5F08FF0BE00E6FD7C00E9FFE8FECE
:01714000222C
:0E717200F88FF0A4FFE5F0CE88F0A42EFE22E8
:10000300EF8DF0A4F9A8F0EF8CF0A428F8EE8DF0B2
:06001300A428FEE9FF2213
:10715200600D782B02715C007830D8FED5E0F82201
:10716200EEC0E07E00127060EFFDEEFCD0E0FE2289
:0C718D00EEC0E07E00127060D0E0FE2238
:03001B0002001EC2
:0300530002005652
:03009B00020071EF
:030000000271ACDE
:0971AC0075817575D000024AB727
:0B004800E5822FF582E5833EF5832260
:0A7199000582D582021583158222BB
:10001E00C0E0C0F0C083C082C0D075D000124A5B71
:0B002E00D0D0D082D083D0F0D0E032E0
:10005600C0E0C0F0C083C082C0D075D000124A5E36
:10006600D0D0D082D083D0F0D0E032C0E0C0F0C093
:1000760083C082C0D075D000124A80D0D0D082D042
:0600860083D0F0D0E0324F
:00000001FF
